:10000000F4C300002AC4000028C4000026C4000075
:1000100024C4000022C4000020C400001EC400004C
:100020001CC400001AC400000C9438320C94203315
:100030000C94ED3112C4000010C400000EC4000086
:100040000CC400000AC4000008C4000006C400007C
:1000500004C400000C94143200C40000FEC300006D
:10006000FCC30000FAC30000F8C30000F6C30000A0
:10007000F4C30000F2C30000F0C30000EEC30000B0
:10008000ECC30000EAC30000E8C30000E6C30000C0
:10009000E4C30000E2C30000E0C30000DEC30000D0
:1000A000DCC30000DAC30000D8C300000501090268
:1000B000A10185020901A1000509190129081500FE
:1000C0002501950875018102050109300931158165
:1000D000257F95027508810609381581257F9501D0
:1000E00075088106050C0A38021581257F95017572
:1000F000088106C0C005010980A101850319012AF4
:10010000B700150126B700950175108100C0050CD8
:100110000901A101850419012AA002150126A002E6
:10012000950175108100C005010906A1018506052C
:100130000719E029E71500250195087501810205D9
:1001400007190029EF1500250195F07501810205B9
:10015000081901290595057501910295017503910D
:1001600001C00660FF0961A1010962150026FF00B8
:100170009520750881020963150026FF00952075FA
:10018000089102C005010906A101050719E029E748
:1001900015002501950875018102950175088101F9
:1001A0000507190029FF150026FF0095067508812F
:1001B000000508190129051500250195057501910E
:1001C00002950175039101C00000000000000000CD
:1001D000000000000000000000000000000000001F
:1001E0000000000000000000000000007E0F00D4AE
:1001F000FFFFFFC7000000780000000000000000C3
:100200002A2B280000000000000000000000000071
:1002100000000029000000002C1E3420212224347C
:100220002627252E362D3738271E1F20212223244E
:1002300025263333362E37381F0405060708090AEA
:100240000B0C0D0E0F101112131415161718191A86
:100250001B1C1D2F3130232D350405060708090A04
:100260000B0C0D0E0F101112131415161718191A66
:100270001B1C1D2F3130354C09025B00030100A00F
:10028000FA09040000010301010009211101000124
:10029000224400070581030800010904010002034C
:1002A000000000092111010001222200070582033C
:1002B00020000107050303200001090402000103D7
:1002C00000000009211101000122B6000705840386
:1002D0002000011201000200000008544D0120011D
:1002E00000010203011C037600690061006C003A02
:1002F00000660036003400630032006200330063A1
:100300000000000E034E00430052002D0038003064
:1003100000000006034D00540000000403090429F6
:100320000000003A003B003C003D003E003F004022
:100330000035001E001F00200021002200230024A1
:100340000025002B0014001A000800150017001CDF
:100350000018000C00390004001600070009000A0C
:10036000000B000D000E00E1002C001D001B00061C
:10037000001900050011001000E000E300E200E4B5
:1003800000650000002C002152E6000000480047F4
:100390000045004400430046004200410027004B56
:1003A000004A002A002C002E0049002D00260000E3
:1003B000004E004D00280030002F004C00130012AA
:1003C0000000000000520000003100340000003343
:1003D000000F0000004F0051002C00E500380050D5
:1003E000003700360001000000010001000100019B
:1003F00000010001000100010001000100010001F5
:1004000000010001000100010001000100010001E4
:10041000000100010001000100010002780100015B
:1004200000010001000100010001000100010001C4
:100430000001000378047805780100010001000143
:100440000001000100530001000000010001000153
:100450000000000100010001000100010001000195
:100460000001000100010001000100010001000184
:100470000001000100000001000100010001000175
:100480000001000100010000000000010000000167
:100490000001000000010001000000010001000156
:1004A0000001000100010001000100010000000145
:1004B0000001000100010001000100010001000134
:1004C0000001000100010001000100010001000124
:1004D0000001000100010001000100010001000114
:1004E0000001000100010001000100010001000104
:1004F00000010001000100010001000100010001F4
:1005000000010001000100010001000100010000E4
:1005100000010001000100000001000100010001D4
:1005200000010001000100010001000100010001C3
:1005300000010001000100010001000000010001B4
:1005400000010001000100010001000100000000A5
:100550000001000000010001000000010001000096
:100560000001000100010001000100010001000183
:1005700000FD377A585A000004E6D6B4460200213E
:100580000116000000742FE5A3E0066302075D007A
:100590003D8889C65436C3174FE4E32F92B46B1FCE
:1005A000E44EA36ABE5F89D37DB09EB5F229AA87C7
:1005B000A34EC569816C2F823FC604B78D04512CB0
:1005C00081C0C73A35DF2F0A0D92F1EA6530A3E00A
:1005D000A47FAA4741779DB6A5FBF402EAE7A411E0
:1005E0000ED1BADC2302DFE09BE588E785A047480F
:1005F000EE83D0FD27C8E7D9B74C849DB3E6EA85E2
:100600001D82217E4A6AED7F2EFE37362DEDB8DA47
:100610004661F8DAB22A98F306EC285752EE7C24A9
:100620000F11C873117A424683CDAF8C889B327903
:10063000539BFD5412593CD440EB9EFEAB8D71A8E8
:10064000463F0CC75478B8FA4D7587BCADD13CC74E
:100650008F2F98723C3FE05DF3CEEAB721C5131BA4
:10066000EFDAE2BF6D01C726FF294739DAEC7D4694
:10067000C9E876FD54D4D4C85DC6DDA02AC0F50310
:100680006A382EFA2A99BCE2854AC307D94231203A
:100690004CCAE48BEEA759F464E7A1FD302574251C
:1006A000E1E598799C55F7D790FF74DFFD6FA69B25
:1006B000D2C9124D8CC8C50E67FBFC1163A6E82D8C
:1006C000F76D491DE5DA3A291DD27749C22752183C
:1006D00035642CA7252A2F9B3DB0607A03CC941457
:1006E000A765DCDB730E63CCB8D304EE54C112A84B
:1006F000B0CEA3DEC20B9979A62439DC655E9E5E7E
:100700003CE8F95C20CA0FDA09749D07C627BA884D
:10071000AED94D7906E5F9522875333929A1F95E2C
:10072000DAF1B11983CF342C2CC9451A07CF0B321B
:10073000BADFA56745CDCE8C42F22B5944B58D2F3B
:100740008BE8918BBC12021A9E83C05D25CA9C80E7
:1007500001F8D5C467CA63CB7FEA4B748A24CE50B4
:10076000F3EF0139F2183B6242673C37155DE26CEA
:10077000A127C3904AC03E541E3293D64B9AE5EA55
:100780006791A11A883B2B4135409D282D89BA736A
:10079000D297645A6E95BC0000DE794305DFC1260E
:1007A000790001A304E40C0000563E5AF9B1C46775
:1007B000FB020000000004595A504F52514A4D4B61
:1007C0004E2A4C2F30B6B7ABACBBBCA9AABDBECF2E
:1007D000D0CDCEDBDCD9DA0D0E0B0F1A05080509DA
:1007E00005071811130408120C0011241FBECFEFC7
:1007F000DAE0DEBFCDBF04B603FE18C080919105DC
:1008000090919205A0919305B09194058730904BFB
:10081000A740B04B59F41092910510929205109296
:10082000930510929405E0E0F8E3099511E0A0E04B
:10083000B1E0E8E5FAE602C005900D92AA3AB107E8
:10084000D9F725E0AAEAB1E001C01D92A139B207AB
:10085000E1F70E94642A0C94AE34D2CB9C019A95A5
:1008600081159F4118F5F32FF270EE27832F8170C9
:10087000732F74706627532F5870442734FF0CC0B1
:100880008295807FEF2B09F08062672B09F08064EE
:10089000452B69F080680895EF2B09F08260672B83
:1008A00009F08460452B19F08860089580E0089570
:1008B000CF93DF93EB01D2DFFE010995DF91CF915A
:1008C00008950C94C9330895982F92959F7024E051
:1008D000911102C020E0982F892F86958695811569
:1008E00011F02E5F982F892F8695820F0895982FEB
:1008F000909580FD08C02D9A91FF07C0469A92FFFF
:1009000006C0479A08952D98F7CF4698F8CF479894
:10091000089580938D05089580938E05089521E0B4
:1009200030E001C0220F8A95EAF780918E05822B74
:10093000F3CF21E030E0A90102C0440F551F8A9592
:10094000E2F7CA01809590918E058923E5CF292F82
:100950009B3090F5893080F590E039E0239F800D41
:10096000911D1124282F277041E001C0440F2A95C2
:10097000EAF723E0969587952A95E1F7FC01EE0FBB
:10098000FF1FE80FF91FE65DFC4F20E030E070E04C
:100990005191DF01CB01022E02C0969587950A94F2
:1009A000E2F7817081958527842385278E932F5FB9
:1009B0003F4F2330310561F70895292F9B3078F59B
:1009C000893068F590E039E0239F800D911D112456
:1009D000682F677023E0969587952A95E1F7FC01CB
:1009E000EE0FFF1FE80FF91FE65DFC4F40E050E0FF
:1009F00080E0219130E0062E02C0369527950A94BA
:100A0000E2F721703327042E01C0220F0A94EAF77F
:100A1000822B4F5F5F4F4330510559F7089580E0B7
:100A2000089590918E0521E030E0F90101C0EE0FAC
:100A30008A95EAF7D90102C0AA0FBB1F6A95E2F7AF
:100A4000EA2B01C0220F4A95EAF7892F8E23E8137B
:100A500003C0892F822B60CF2095822F8923FBCF63
:100A60008091D8029091D702981301C008958F5FAA
:100A70008770FACF9091D904809589238093D90407
:100A8000282F2770211110C0891771F090919005BF
:100A900092FF0AC08695869586954BDF1092D90401
:100AA0001092DB041092DA0408959091D604982BEA
:100AB0009093D6040895982F90958091D604892319
:100AC0008093D60408958091D504811531F0109259
:100AD000D5041092DD041092DC040895803E910547
:100AE000D9F1C8F48133910509F482C048F4893200
:100AF000910509F472C08A32910509F480C0089505
:100B000089339105E9F082389105D1F0853391055B
:100B100009F45EC00895843E9105D9F148F4823EFF
:100B2000910539F1833E910549F181EE90E00895F8
:100B3000863E9105C9F1873E910509F43EC00895AE
:100B400020918F052370211164C02091900523FF0F
:100B500014C089E290E0089520918F0520FD45C0E2
:100B60003091900530FF09C024FD24C083EE90E051
:100B7000089520918F0522FDF7CF089520918F05CC
:100B800022FD44C03091900530FD43C024FFF5CFD5
:100B900011C02091900521FFF0CF80918F0584FD39
:100BA00009C087EE90E0089520918F0523FFE5CFDF
:100BB00024FFF7CF80E090E0089520918F0523FD7A
:100BC0002BC03091900531FFE1CF84EE90E0089585
:100BD00020918F0525FFD1CFBCCF20918F0525FD1A
:100BE0001EC02091900523FFC8CF89E390E00895AF
:100BF00020918F0526FFC1CF8AE290E008952091D1
:100C00008F0526FFBACF81E390E0089582EE90E051
:100C1000089580EE90E0089586EE90E0089585E3D3
:100C200090E0089590918F0592FF10C041E0282F29
:100C30002471243009F040E031E0282F2871283059
:100C400009F030E0431711F02CE0822793FF10C029
:100C500041E0282F2471243109F040E031E0282FB1
:100C60002871283109F030E0431711F02CE0822779
:100C70003091900530FF10C051E0282F21712130B4
:100C800009F050E041E0282F2871283009F040E0B9
:100C9000541711F029E0822731FF10C041E0282FBE
:100CA0002171213109F040E031E0282F28712831ED
:100CB00009F030E0431711F029E0822794FD877E88
:100CC00008951F93CF93DF9309DFEC01811522E58F
:100CD000920708F052C0811540E5940708F0CDC096
:100CE000803E910520F58D3C910508F0A1C0883A21
:100CF000910570F4853A910508F097C0813091050F
:100D0000B9F10497813A910598F1C0E0D0E030C084
:100D1000885A91094B97C8F7C85AD0E0CC0FDD1F0D
:100D2000C25CDE4F0990D881C02DD46421C08115EA
:100D300050E49507B0F4C11580E2D80708F0B3C0BD
:100D4000C83ED105A8F0CE019A9581159F41E8F6DD
:100D50008D2F68DF182FCE019927C0DEEC01D12B33
:100D600007C09927BBDECC27DF70C82BD92BD06AF0
:100D7000CE01DF91CF911F910895803842E594070D
:100D8000C8F5803652E5950708F05BC0C03482E5AF
:100D9000D807D0F4C03292E5D90708F04BC08C2FA9
:100DA0008695869520E2829FC0011124C37021E0C0
:100DB00030E0A90102C0440F551FCA95E2F7EA01CD
:100DC000C82BD92BDD68D4CF8C2F8695869587705C
:100DD00050E2859FC0011124C37021E030E0A901D9
:100DE00002C0440F551FCA95E2F7EA01C82BD92B60
:100DF000DC68BECF803C52E5950758F48F71C03A4D
:100E0000D245A0F590E0982F8827EC01C46FD06AF6
:100E1000AFCF805C9245809708F077CFDC2FCC274E
:100E2000CC27DF71C06FD06AA3CFA497D064A0CFC6
:100E3000D0659ECFCF71D0E0DC2FCC27C16FD06AB8
:100E400097CF86958695877020E2829FC0011124F6
:100E5000C37021E030E0A90102C0440F551FCA95BC
:100E6000E2F7EA01C82BD92BDA6882CFDBDEC82F84
:100E7000D0E0DC2FCC27D0627BCF8F71D3DE93E024
:100E8000CC0FDD1F9A95E1F7CC27DF70282F30E0DB
:100E900084FF05C050E1859F900111243327C22BA8
:100EA000D32BD06965CF8D2F8F71BCDE182FCE016B
:100EB000992714DEEC01D12BDECF80E00895F89461
:100EC000E82FE295EF70F0E041A18F7021E030E073
:100ED000B90102C0660F771F8A95E2F7CB01962F02
:100EE0009095942391A392A1892B82A3789408953D
:100EF000A0E0B0E0EEE7F7E00C940334863080F534
:100F000081112FC0909180009F7D9093800020914F
:100F1000860030918700A82FB0E00E94E03325E0E2
:100F200030E040E050E00E94A13369017A018091F5
:100F30008600909187006CE070E00E947A3362171F
:100F4000730798F0C90169E070E00E947A337093EA
:100F50008B0060938A00CDB7DEB7E8E00C941F34B5
:100F600085E0909180009062D0CF80918600909132
:100F700087000091860010918700209186003091B3
:100F80008700C6E0D0E0BE010E947A33C60ED71EAD
:100F9000E11CF11C85E0CC0CDD1CEE1CFF1C8A95CD
:100FA000D1F7C801BE010E947A3340E050E0260F1D
:100FB000371F411D511DC701B6010E94A1336901B0
:100FC0007A01E0918600F0918700CA01B9010E9480
:100FD0006B339B01AC01DF010E94EF339B01AC013D
:100FE000C701B6010E946B332FE0969587957795E0
:100FF00067952A95D1F720918600309187002617B2
:1010000037071806190608F0A2CF60918600709184
:1010100087009DCF982F990F990F990F2091C403A6
:101020002770922B9093C40321E0983008F420E0BD
:101030009091C40320FB90F99093C40359CF81157C
:101040002CE7920741F42091A4023091A502232BB2
:1010500011F480E090E00895EEE4F4E080E090E0A8
:1010600069EC78E24CEE58E22EE539E2778366834C
:1010700051874087338722879787868701967096A6
:101080008830910599F70895FB01811520E29207B8
:1010900028F4811541E0940738F408959C013052FA
:1010A0002115304348F00895392F94FF02C032953E
:1010B000307F2081232B208399270895462B22FF00
:1010C0000FC0982F92959F708F70892B962F9295B5
:1010D0009F706F70692B942F92959F704F70492B62
:1010E000982F9623961309C050E04095509590E0B4
:1010F0004823592381E0452B09F080E008951092A0
:101100001F0510921E05EEEDF4E08581811102C0ED
:1011100014821682379685E0E631F807B1F7089514
:10112000AC013091210560912005232F621301C08D
:101130000895822F90E0FC01EE0FFF1FEA5EFA4F48
:101140000190F081E02DE417F50791F467E0649FCA
:10115000F001659FF00D1124E252FB4F41E0448302
:101160002313E6CF01968370992780932105089574
:101170000196282F2370DACFFC0184818623811108
:101180000AC082818115B9F06823908593FF05C05C
:1011900081E061110FC080E00895282F22952F7003
:1011A0008F70282B962F92959F706F70962B81E0F1
:1011B0002913F1CF089581E008950F931F93CF93E2
:1011C00001E010E0082E01C0000F0A94EAF7C09178
:1011D000D4049C2F9023911115C09091D904969519
:1011E00096959695891306C01092D9041092DB0447
:1011F0001092DA0494DBC027C093D404CF911F91DE
:101200000F91089596DBF7CF282F35EB2303C0010C
:10121000112497FF04C080589109892F08958058A0
:101220009F4FFBCF8091530380FD14C081FD14C0FC
:1012300082FD16C080915203811581F08E3180F4B9
:1012400020E5829FC00111246EE170E00E948E3380
:10125000862F089584E1089588E2089588E008952E
:1012600080E508958091530380FD17C081FD17C06C
:1012700082FD19C080915103811599F0883298F44C
:1012800028E0829FC001112468E270E00E948E3342
:101290006115710551F0862F089562E0FCCF64E07E
:1012A000FACF61E0F8CF68E0F6CF81E00895909141
:1012B000AF0389029001112437FF03C08093AF036D
:1012C00008952F3731051CF4980F9093AF030895BC
:1012D0009C0180E090E0F901E80FF91FE491E4132C
:1012E00007C091E08927F901E80FF11D8491089565
:1012F0000196861780F380E00895FA01309709F08F
:1013000009950895E091CD02F091CE02309739F021
:101310000190F081E02D309711F00995089580E05B
:101320000895A3E0B0E0E7E9F9E00C9409349C01EA
:101330008091F2019091F30182179307B1F03093FD
:10134000F3012093F201E091CD02F091CE023097AB
:1013500061F00084F185E02D309739F083E08983D6
:101360003B832A83CE01019609952396E2E00C94F3
:101370002534A3E0B0E0EFEBF9E00C9409349C01D4
:101380008091F0019091F10182179307B1F03093B1
:10139000F1012093F001E091CD02F091CE0230975F
:1013A00061F00084F185E02D309739F084E0898385
:1013B0003B832A83CE01019609952396E2E00C94A3
:1013C000253490910E01913091F0AEEAB1E0EFEF4B
:1013D00090E02D91821751F0EF3F19F4211101C0D7
:1013E000E92F9F5F9630A9F7EF3FC9F408959091D8
:1013F0008F0597FFEACFE82FE695E695E695803FC3
:10140000A8F7F0E0EC54FE4F877021E030E001C017
:10141000220F8A95EAF78281822B828308950E2E0D
:10142000000CFF0BE455FE4FF8CF90910E01913068
:1014300021F490918F0597FD0CC0EEEAF1E09191B7
:10144000891302C0DF011E9251E0E43BF507B9F7B2
:101450000895E82FE695E695E695803FC8F7F0E019
:10146000EC54FE4F877021E030E0A90102C0440F28
:10147000551F8A95E2F7CA0180959281892382835C
:10148000089580910D0108952FB7F8948091EC0193
:101490009091ED01A091EE01B091EF012FBF089561
:1014A000CF93DF93C091D6048091D804C82B80914C
:1014B000D5048115F1F0E8DF2091DC043091DD04E2
:1014C000821B930B8838934108F0FDDAD091D50444
:1014D00080910E01813021F480918F0587FD13C02A
:1014E00086E02EEA31E090E0815088F49111EBDA49
:1014F000CD2B8091CA0380958C239091C903892BB1
:10150000DF91CF9108958EE126EB31E0ECCFF90128
:1015100041919F01411541F39F5FE6CF962F2091A6
:10152000900522FF0EC0682F660F660F660F692BAD
:101530006093D904F4D9A8DF9093DB048093DA0494
:101540000895EDC99091D504292F2823211559F02C
:10155000809589238093D504811531F095DF8093A0
:10156000DC049093DD04089580E090E0F8CF8CDFF8
:101570002091560330915703232B211521F080939E
:101580008702909388022091580330915903232BAE
:10159000211521F08093850290938602E091CD027F
:1015A000F091CE02309759F00680F781E02D309708
:1015B00031F082E08093540384E593E00995089527
:1015C000611509F441C0E3E3E80FE33148F4F0E0CA
:1015D000E055FB4C0C94C33325DE81958093570373
:1015E000C6CF20DEFBCF1EDE819580935603F8CF59
:1015F00019DEFBCF37DE80935803F2CF33DE8195BF
:10160000FACF30DE819580935903EACF2BDEFBCFF2
:10161000815D990B21E030E001C0220F8A95EAF745
:1016200080915503822B80935503DACF8091530329
:10163000816080935303D4CF809153038260F9CFAC
:10164000809153038460F5CF409156038D3C59F44B
:101650008091570387FF0DC010925703411559F42D
:101660001092520308C08E3C81F4809157031816E3
:101670009CF3411581F08091580390915903892B77
:101680008111AECF10925103ABCF8F3C41F447FF95
:10169000F0CF10925603809157038115E0CF803D23
:1016A00019F41416B4F3E5CF90915803893D29F449
:1016B0001916FCF610925803DCCF8A3D19F497FFF7
:1016C000D8CFF8CF909159038B3D29F497FFD1CF14
:1016D00010925903CECF8C3D19F41916CCF3C9CF13
:1016E0009FE2980F983090F4815D990B21E030E0F3
:1016F000B90102C0660F771F8A95E2F7CB0180958A
:1017000090915503892380935503B3CF8D3D31F4D8
:10171000809153038E7F80935303ABCF8E3D21F492
:10172000809153038D7FF7CF8F3D09F0A2CF809139
:1017300053038B7FF0CF2FB7F8946091EC01709139
:10174000ED018091EE019091EF012FBF0895CF92AE
:10175000DF92EF92FF92CF93DF93D82FC92FC090E3
:101760004804D0904904E0904A04F0904B04E3DF31
:101770006C197D098E099F09643F714081059105AF
:1017800010F1D9DF6B017C0182E390E0A0E0B0E0D2
:10179000C0928102D0928202E0928302F09284028F
:1017A00080937D0290937E02A0937F02B09380028B
:1017B000D0934604C0934704DF91CF91FF90EF9000
:1017C000DF90CF90089584EF91E0A0E0B0E0E0CF0B
:1017D000FC019B018091E2019091E301861797073C
:1017E00040F0672B29F48091E8008E778093E80021
:1017F000C90140E0009741F4411106C08091E80022
:1018000082FF2FC080E008952091A6022115A9F142
:101810002530A9F12091E80023FD2DC02091E8009A
:1018200022FDECCF2091E80020FFE4CF3091F300BF
:101830002091F200009719F02830310558F041E06E
:101840002830310509F040E02091E8002E77209300
:10185000E800D0CF41914093F10001972F5F3F4FB7
:10186000E9CF8091A602811541F0853041F0809149
:10187000E80083FFC3CF81E0089582E0089583E00C
:1018800008958091DC0187FF13C08091E80082FFFA
:1018900006C08091E8008B778093E80008958091DE
:1018A000A6028111F2CF08958091A6028115D9F385
:1018B0008091E80080FFF8CF8091E8008E77ECCF30
:1018C0002091E4003091E50095E6A9012091EC001B
:1018D000822F817020FF06C08091E80080FF06C043
:1018E00080E008952091E80022FD1AC08091A602B0
:1018F000811589F0853089F08091EB0085FD0FC05E
:101900002091E4003091E50042175307F9F29A95CF
:10191000E1F684E0089582E0089583E0089581E08F
:101920000895E8EDF0E080818E7F80831092E200E0
:101930001092DA001092E100A0EEB0E08C9181608C
:101940008C9380818F77808319BCA7EDB0E08C9158
:101950008E7F8C9380818F7E80831092DB0108952F
:10196000E091CD02F091CE02309739F00284F385F8
:10197000E02D309711F060E209950895982F90932B
:10198000E900891771F07091EC002091ED00509101
:10199000F00021FD09C09F5F973089F78093E9002F
:1019A0000895762F242F50E03091EB003E7F309346
:1019B000EB003091ED003D7F3093ED003091EB0076
:1019C00031603093EB007093EC002093ED00509366
:1019D000F0002091EE0027FDDECF0895A0E0B0E0FA
:1019E000E4EFFCE00C940334C8EDD0E088818F7EF6
:1019F0008883E7EDF0E080818160808384E082BFAE
:101A000081E08093DB0188818E7F888302EE10E085
:101A1000F80110821092DA0081EEC82ED12CF60166
:101A2000108288818F778883888180688883888105
:101A30008F7D888319BC1092A6021092DA01109251
:101A400065021092D90190EEE92EF12CF701808108
:101A50008B7F808388818160888342E060E080E0C2
:101A60008DDFF60180818E7F8083F8018081816027
:101A70008083808188608083F70180818E7F80836E
:101A8000888180618883CDB7DEB7E8E00C941F348D
:101A9000E091D8029091D70229E0E91302C080E0DA
:101AA0000895AE2FB0E02E9FF0011124E752FD4FB4
:101AB0003181361306C03081381303C035813413A9
:101AC00004C0FD013196E770E8CF81E0089581E020
:101AD0008093E00080E28093D8001092C9008FE1EB
:101AE0009EE40197F1F700C0000087E090EBDC0175
:101AF0008093910590939205A0939305B0939405DC
:101B000088E19CE00FB6F894A895809360000FBE22
:101B100090936000FFCF0F931F93CF93DF938B01C0
:101B2000EA019091A602943051F58093E9008FEF7D
:101B30009091E80095FD06C095ED9A95F1F70000AB
:101B40008A95B1F78091E80085FF19C0B9DE81114F
:101B500011C08091E80085FD06C08091E8008E7775
:101B60008093E800F3CFF80181918F018093F10019
:101B7000219779F78091E8008E778093E800DF91D4
:101B8000CF911F910F910895792F603229F440E28F
:101B900050E0682F82E0BFCF0895CF93DF93D82F16
:101BA000C92F48E050E0682F792F81E0B4DF88E04A
:101BB000ED2FFC2FA4EEB1E001900D928A95E1F794
:101BC000DF91CF910895BC0140E250E084E0A3CFC3
:101BD000BC0146E050E084E09ECFBC0143E050E011
:101BE00084E099CF9091900592FB222720F9281745
:101BF00079F080FB92F99093900560918F05709138
:101C0000900584E090E00E94933482E00C943A05C1
:101C10000895FC01608186E090E00C9479341F9374
:101C2000CF93DF93962F122F632F8330D8F49B30FE
:101C3000C8F44930B8F4C42FD0E0CC0FDD1F22E146
:101C4000929FC00DD11D112496EC899FC00DD11D0E
:101C50001124CE0189960E947934612FCE018A9693
:101C60000E947934DF91CF911F91089580910E01E8
:101C7000813061F580918F0587FF28C011DC80934A
:101C8000B50140E250E06DEA72E084EB91E00E9421
:101C90003934892BD1F080E2E4EBF1E0ADEAB2E037
:101CA00001900D928A95E1F7E091CD02F091CE027C
:101CB000309759F00480F581E02D309731F086E0BF
:101CC0008093B40184EB91E009950895E9DB80935A
:101CD000AC0148E050E06FEC72E08CEA91E00E94C9
:101CE0003934892B91F388E0ECEAF1E0AFECB2E013
:101CF00001900D928A95E1F7E091CD02F091CE022C
:101D0000309719F30280F381E02D3097F1F28CEADD
:101D100091E0DACF811519F00E945505A7CF0895FB
:101D2000811531F09091D804892B8093D8049ECFEF
:101D30000895CF93C82F8115C1F08CEF8C0F813A95
:101D400080F580910E01813021F480918F0587FD0F
:101D50000EC0EEEAF1E08191C817F9F021E0E43B12
:101D6000F207C9F78C2F2DDB81DFCF910895EC2F7F
:101D7000E695E695E695F0E0EC54FE4F828190E022
:101D80004C2F477021E030E002C0220F331F4A95EC
:101D9000E2F782239323892B29F38C2F46DB66DF1E
:101DA000E1CF80E28C0F883048F4C77081E001C039
:101DB000880FCA95EAF70E945505D6CF8BE58C0FA0
:101DC000833030F42C2F2452330BC901AADACDCF43
:101DD000E8E5EC0FEB3148F4F0E0EE0FFF1FEC58B4
:101DE000FE4F80819181C5DAC0CF83E38C0F8331B0
:101DF00008F0BBCF61E08C2FE3DBB7CFCF93DF934D
:101E0000EC01805E9109089720F060E97EE0209760
:101E100011F46AE87EE0CE010E9458048C2F89DF1D
:101E2000DF91CF910895811541F19CEF980F913A80
:101E300010F4FBDA1BCF90E2980F983050F48770C3
:101E400091E001C0990F8A95EAF7892F0E945B05FE
:101E5000F1CF9BE5980F933018F480E090E061CAD1
:101E600098E5980F9B3118F480E090E082CA93E3E4
:101E7000980F933110F460E0A3CB08951F93CF9394
:101E8000DF93182FEB0155DF209731F4812FCBDF43
:101E9000DF91CF911F9108958FE99FE00197F1F7AE
:101EA00000C000002197F0CF811519F00E945B055A
:101EB000DDCE0895811539F080959091D80489235D
:101EC0008093D804D3CE08958091C503811521F065
:101ED00082E2F0DF1092C50308951092D60480913B
:101EE0000E01813011F580918F0587FF1EC0E6EB52
:101EF000F1E08EE1DF011D928A95E9F780E090E044
:101F000010DA80E090E035DA1092D804AFDE86E097
:101F1000E4E5F3E0DF011D928A95E9F710925203A0
:101F2000109251031092530322CBEEEAF1E086E0C7
:101F3000E1CFD3DF2FEF84E39CE02150804090403D
:101F4000E1F700C0000088E19CE00FB6F894A89586
:101F5000809360000FBE90936000FFCFAAE2B0E0D4
:101F6000E4EBFFE00C9408348CED91E0FC01019669
:101F70002091F100208321E0843E9207B9F78091FF
:101F8000DD01893009F457C0C8F4823009F4B2C0C9
:101F9000833009F482C0813081F18091E80083FFB1
:101FA000E6C08091DC019091DD019A3008F0DFC03D
:101FB000E92FF0E0ED53FB4C0C94C3338A3009F465
:101FC00089C08B3051F78091DC01813231F78091EB
:101FD000E0019091E101892B01F78091E800877F72
:101FE0008093E8004EDC81E09091DE01911101C008
:101FF00080E080930E0171DFD0CF8091DC01813AC7
:1020000061F68091E800877F8093E8008091E0018D
:102010009091E101892B59F060E080E090E070E060
:10202000D7DB8091E8008B778093E800B6CF68E03B
:1020300084EE91E0F4CF8091DC01813209F0ADCFE4
:102040008091E0019091E1018D7F892B09F0A5CF6E
:102050008091E800877F8093E8008091E80082FF0C
:1020600017C09091F3008091F200029731F48091B3
:10207000F100813011F0863021F48091F1008093DD
:102080000D018091E8008B778093E800FADB85CF23
:102090008091A6028111E1CF80CF8091DC01813A4D
:1020A00009F07BCF8091E0019091E101892B09F04B
:1020B00074CF8091E800877F8093E8008091E800EA
:1020C00080FFFCCF80910E018093F1008091E800A9
:1020D0008E77DACF8091DC01813209F05ECF80917A
:1020E000E800877F8093E800CCDB8091DF0180935C
:1020F0000C0153CF8091DC01813A09F04ECF8091E1
:10210000E800877F8093E8008091E80080FFFCCFA3
:1021100080910C01D9CF803889F0823841F58091C7
:10212000E0018F70873018F58093E9008091EB0013
:1021300085FB882780F91092E90006C0809165022E
:10214000880F9091D901892B9091E800977F909307
:10215000E8008093F1001092F1008091E8008E7702
:1021600023C0811116C08091DE01813009F1809178
:10217000E80083FF0AC08091E800877F8093E80031
:102180008091EB0080628093EB00AA96E3E00C94D0
:102190002434823061F78091DE01811581F0109244
:1021A000E9008091E800877F8093E8006ADBDFCF59
:1021B00081E0933009F080E080936502F0CF809158
:1021C000E0018F702FEF280F263088F68093E9000A
:1021D0002091EB0020FFE3CF933031F48091EB00AE
:1021E00080628093EB00DBCF9091EB009061909345
:1021F000EB0021E030E0A90102C0440F551F8A9591
:10220000E2F74093EA001092EA008091EB008860C8
:10221000E8CF8111ACCF1091DE011F778091E300F0
:102220008078812B8093E3008091E800877F809302
:10223000E80027DB8091E80080FFFCCF8091E3007D
:1022400080688093E30083E0111101C082E08093F5
:10225000A6028DCF8058823008F089CF8091DE01B0
:102260009091DF018C3D53E0950791F583E08A83DF
:102270008AE289834FB7F894DE01139620E03EE0AE
:1022800051E2E32FF0E050935700849120FF03C008
:1022900082958F703F5F8F708A30C0F0895C90E0CC
:1022A0008D939D932F5F243161F74FBF8091E8009C
:1022B000877F8093E8006AE270E0CE01019688DAB9
:1022C0008091E8008B778093E80051CF805DE7CF65
:1022D000292F33272330310509F44EC078F52130FA
:1022E000310509F488C08BE590E0E8E7F2E02230A0
:1022F000310509F03CCF2091E800277F2093E800CA
:102300002091E2013091E3018217930708F49C01C8
:1023100040E02115310509F073C0411171C0809171
:10232000E80082FDCDCF8091A602811549F285306B
:1023300039F28091E80083FFF2CFC2CF8091E001B3
:102340009091E1012132310509F446C02232310574
:1023500009F00DCF8330910508F009CFFC01EE0F95
:10236000FF1FE25EFE4F0190F081E02D855E9E4FE3
:10237000DC018C9190E010C09C013327823021F168
:102380002330310568F4232BB9F4EBE1F3E0E49159
:102390008E2F90E0EBE1F3E0009709F4E8CEABCFAD
:1023A0002330310509F0E3CEE5EEF2E0E4918E2F23
:1023B00090E0E5EEF2E0F0CFE3E1F3E0E4918E2F80
:1023C00090E0E3E1F3E0E8CFE3E0F3E0E4918E2F87
:1023D00090E0E3E0F3E0E0CF8330910508F0C7CE72
:1023E000FC01EE0FFF1FEC5DFE4F0190F081E02D30
:1023F00089E090E080CF82E190E0E3EDF2E07BCFF6
:102400008091A602811509F45BCF853009F458CF7D
:102410008091E80083FD54CF8091E80082FD7FCF5A
:102420008091E80080FF75CF9091F3008091F200D9
:102430002115310519F08830910550F041E00897D9
:1024400009F040E08091E8008E778093E80061CF4A
:1024500044914093F1003196215031090196E8CF23
:10246000803809F084CE8091E800877F8093E8006F
:102470008091DA018093F10070CE811178CE1091B5
:10248000DE01123008F073CE8091E800877F8093E0
:10249000E8001093DA01F5D91115D9F084E08093A2
:1024A000A60242E061EC81E069DA42E261EC84E09C
:1024B00065DA42E261EC82E061DA42E260EC83E0FC
:1024C0005DDA8091A602843051F482E080930F019E
:1024D0004ECE8091E30087FDE1CF81E0E0CF81E047
:1024E000F5CFCF93DF93EC014A855B856E857F85C1
:1024F0000E947D099B8190958091D80489238093C7
:10250000D8048C810E945B05B1DB86E0FE0111924C
:102510008A95E9F7DF91CF910895CF93DF93EC018E
:102520008D8181FD13C082608D838091D8049B8151
:10253000892B8093D8048C810E94550597DB4885B0
:1025400059856E857F85CE010E947D091092CF044A
:102550001092CE048D8180FD02C0CE01C2DFDF91DA
:10256000CF9108951F93CF93DF93182FA091440428
:10257000B0914504109709F448C010924704109296
:1025800046041092CA031092C9031696CD91DC91AD
:102590001797CE019A9581159F4108F4D07ED1E01E
:1025A000C11101C0D0E01996ED91FC911A973097B6
:1025B00031F01B966D917C9180E00995D823D1155F
:1025C00039F08CEF8C0F813A20F58C2F0E94150A80
:1025D0001115A1F0E0914404F0914504808584FD3B
:1025E0000DC080914304811549F0808191819C0147
:1025F000215031092F333E4708F4A9D837DB109218
:1026000045041092440410924304DF91CF911F912E
:1026100008952CDB8C2F07DCDBCF86E090E00E9456
:102620005D348093C40382FD06C08DE28093C403B1
:1026300084EC93E0EEDA8091C403803320F087705D
:1026400088628093C4039091C403892F817090FFA6
:1026500004C0892F8695869586950C9478070F93EC
:102660001F93CF93DF93833030F56B3020F54930E3
:1026700010F5C42FD0E0CC0FDD1F22E1629FC00D0A
:10268000D11D112436EC839FC00DD11D1124CE0124
:1026900089960E945D34082F10E0102F0027CE018C
:1026A0008A960E945D349801282BC901DF91CF9151
:1026B0001F910F91089580E090E0F8CF462F672F8B
:1026C0002091A9023091AA02232B81F4703F39F4A2
:1026D000403F61F48091A7029091A80208957B3059
:1026E00028F4493018F4833008F4B9CF80E090E042
:1026F0000895A0E0B0E0EFE7F3E10C9404347C012E
:1027000000918E0580918D05082BC2E0D0E010E08D
:10271000C8010C2E02C0959587950A94E2F780FDBA
:1027200009C02197A8F7D12C8D2DCDB7DEB7E7E0F2
:102730000C942034DC2EB7018C2FC0DF0E94610680
:10274000019779F3F1CF0F931F93CF93FC0187810A
:102750009085009789F4858100811181811581F030
:10276000611571F0C801C5DFC82F682FC8010E942C
:10277000A704B8018C2FA2DFCF911F910F9108956C
:10278000C8010E94DD04C82FF4CFCF93DF93D82F68
:10279000C92FAFDF6D2F7C2F91DF0E946106DF9183
:1027A000CF910895FC0184818115B1F087819085D6
:1027B0000097A1F00E946106282F92959F70963095
:1027C000B9F080F4925F9F70923030F4203FD1F0E6
:1027D00058F481E0283E58F080E00895808191818E
:1027E000D4DFEACF9A5FEFCF81E0243FA9F70895C5
:1027F00091E0813F09F090E081E0283E08F080E020
:10280000892B089581E00895382F292FCB01A32F1C
:10281000B22F85369105A105B10520F485569C4F50
:102820000C945D3480E0089585E290E00E945D3470
:10283000873089F486E290E00E945D34893659F44D
:1028400087E290E00E945D3491E0893609F090E0E3
:10285000892F8170089580E0FCCFAAE0B0E0E3E327
:10286000F4E10C94FE33C090A402D090A50281E064
:1028700090E09093A5028093A402812C912CE12CEE
:102880005401F12C14C0F80125913591472D6F2D7D
:102890008E2DC5D90E5F1F4F739489E07812F3CF48
:1028A00099E0A90EB11CF394EBE0FE1639F0850116
:1028B000000F111F015E1C4F712CE5CFE394F3E66E
:1028C0008F0E911C83E0E812DBCF1A8219821C82E2
:1028D0001B821E821D8218861F8288EC90E09A87D8
:1028E00089870BE712E0FE0131967F014AE050E054
:1028F000B801C7010E949734065F1F4F0B3CF2E0FE
:102900001F07A1F78AE0F70111928A95E9F74AE0DB
:1029100050E0B801C7010E949734065F1F4F0B318A
:10292000F3E01F07A1F789E0F70111928A95E9F713
:102930008FEF9FEF9E838D8387E08A874AE050E088
:10294000B801C7010E949734065F1F4F0B36F3E0B2
:102950001F07A1F786E0F70111928A95E9F746E093
:1029600050E0B801C7010E9497340A5F1F4F0B392E
:10297000F3E01F07A1F7D092A502C092A4022A9605
:10298000EDE00C941A34AAE0B0E0E9ECF4E10C9428
:102990000334E6EFF1E080E5DF011D928A95E9F767
:1029A000EEEDF4E088E3DF011D928A95E9F786EF0A
:1029B000C82E81E0D82E7F010BEC12E0F701D18206
:1029C000C0824AE050E0B801CE0101960E944D3429
:1029D00088E0FE013196D60101900D928A95E1F7CB
:1029E00089859A85D70113969C938E931297BAE0A6
:1029F000CB0ED11CE7E0EE0EF11C065F1F4F0B3132
:102A0000F3E01F07D9F62A96E8E00C941F34AAE0F9
:102A1000B0E0EDE0F5E10C9401340BEC13E08BE158
:102A2000E82E83E0F82E97E0B92E25EFC22E21E0A4
:102A3000D22EAA24A3944AE050E0B701CE01019619
:102A40000E944D34F8013896DF018B2D1D928A9536
:102A5000E9F789819A81D80111969C938E938F8191
:102A600012968C9312978D8113968C931397888569
:102A700014968C931497898515968C9315978B8152
:102A80009C8117969C938E9316978A8587FD04C028
:102A90001E96DC92CE921D9780FF02C0F801A086A0
:102AA00081FF07C0D80118969C91189792601896DC
:102AB0009C9382FF04C0F80190859460908783FF07
:102AC00007C0D80118969C911897986018969C9307
:102AD00084FF04C0F80190859061908785FF07C04E
:102AE000D80118968C911897806218968C93BAE04A
:102AF000EB0EF11C015F1F4FEBE6EE16E3E0FE0666
:102B000009F099CF2A96EAE00C941D34A6E0B0E0D3
:102B1000ECE8F5E10C94043404E613E08BE6E82ECF
:102B200083E0F82E98E0D92E46E050E0B701CE01C0
:102B300001960E944D34F8018D2D11928A95E9F786
:102B4000B8016C5F7F4F89819A810E944408F80127
:102B500091838083B8016B5F7F4F8B819C810E9442
:102B60004408F801938382838D8186838E818783D5
:102B7000F6E0EF0EF11C085F1F4F8BE9E81683E0CB
:102B8000F80691F62696E7E00C942034282FCB0126
:102B9000283070F44AE0249F90011124B90165584F
:102BA0007D4F4AE050E00E944D3480E090E008956F
:102BB0008FEF9FEF0895AAE0B0E0E1EEF5E10C940D
:102BC00009349C0197558115914068F4BE016F5FEF
:102BD0007F4F822FDBDF892B31F489859A852A96F6
:102BE000E2E00C94253488EC90E0F9CFA0E0B0E06E
:102BF000ECEFF5E10C940434162FD72FC42FD22E0E
:102C00008115A1F04093D2040E94440A9093D80108
:102C10008093D701C77081E001C0880FCA95EAF799
:102C200079D8CDB7DEB7E7E00C9420349091D20488
:102C3000491335C0E090D701F090D8010E94440AB2
:102C40009C012E193F097901812F9D2FB4DFE816D1
:102C5000F90628F5D0E2DD0DCD1591F0C77011E031
:102C6000812F01C0880FCA95EAF71ED9D83040F4E9
:102C70008D2D877001C0110F8A95EAF7812F4AD8F0
:102C800060E070E0802FFAD8D83058F62D2D2770EC
:102C900081E001C0880F2A95EAF706D9C2CFC77034
:102CA00081E001C0880FCA95EAF7F7CFA0E1B0E054
:102CB000ECE5F6E10C94FB33FE01319680E1DF0197
:102CC0001D928A95E9F707E010E09BE9A92E93E0B1
:102CD000B92E25E6422E512C612C712C4F01730127
:102CE0006201B1E14B165104610471041CF080E1F2
:102CF000C82ED12CA601B501C4010E946A34AC0CC7
:102D0000BD1C0D2C000CEE08FF084C185D086E0869
:102D10007F080150104019F76096E0E10C941734D9
:102D20006FEF85E290E00E9479346FEF86E290E0E9
:102D30000E9479346FEF87E290E00E94793460E07E
:102D400088E290E00E94793488DDB0DF67E085E2B8
:102D500090E00E94793469E686E290E00E9479343E
:102D600069E687E290E00C947934A0E0B0E0EBEB08
:102D7000F6E10C940234EC018881811511F1813067
:102D800009F046C08981813051F48A81239660E53B
:102D900070E0893311F060E070E070D8EDCF8230E0
:102DA00029F48A8123960E94990EE6CF833021F47C
:102DB0008A81239638D8E0CF843041F02296811161
:102DC000DBCFCDB7DEB7E9E00C941E348A812396C1
:102DD00020E030E09AE0682F6053770BAB016A3057
:102DE000710560F02115310551F3EFE9FFE03197EE
:102DF000F1F700C0000021503109F4CF929FB001DB
:102E0000939F700D11249A01260F371F8991E3CFEC
:102E1000E82FF0E0E850FE4FB490282F2695269535
:102E2000269530E0F901E851FE4FE4908770F12CCF
:102E3000082E02C0F594E7940A94E2F7E0FAEE2433
:102E4000FF24E0F8F901E852FE4FC490D12C082E7F
:102E500002C0D594C7940A94E2F7C0FACC24DD24CA
:102E6000C0F8F901E853FE4F049110E002C0159537
:102E700007958A95E2F701701127E114F10419F022
:102E800081EE0E94990EC114D10419F086EE0E94C1
:102E9000990E60E070E08B2D0E943E0FC114D104AA
:102EA00019F086EE0E94130FE114F10419F081EE7F
:102EB0000E94130F0115110529F060E070E08CE20B
:102EC0000E943E0F219658CFACE0B0E0EAE6F7E171
:102ED0000C94F9337C01DC0114968C91811509F472
:102EE0001AC161E0C7012FDC8C01F70185818115D2
:102EF00021F18091CE049091CF040097F1F0081752
:102F00001907D9F0FC01FF27887F9927892B09F041
:102F10004BC0B4E0EE0FFF1FBA95E1F7E25BFB4F49
:102F200085818460858311830083CF01F6DA109256
:102F3000D80461E0C70107DC8C018091B9038111DD
:102F40003AC0D70115968C91811509F499C00115E5
:102F5000B0E51B0708F07FC00115E0E21E0708F08E
:102F6000DEC00115F7E01F0731F108F5C801805EEA
:102F70009109089700F13091D6048091D8042091EE
:102F8000D50499E0F701A5EAB3E001900D929A9576
:102F9000E1F71093AD030093AC031092AF03832BC2
:102FA000822B8093A40307C0E0E0F0E0B9CF0115C5
:102FB0003FE0130701F7F70185818111ADC1680179
:102FC00057E5D51AC11481E0D80608F0C4C26AEBEF
:102FD00073E08C2DDBDD892B31F5C601E4E0880F31
:102FE000991FEA95E1F7FC01E25BFB4F228121305A
:102FF00009F0C2C22091BA033091BB03232B99F090
:103000002091BC033091BD03232B69F02091BE03B6
:103010003091BF034091C0035091C103242B352B45
:10302000232B09F4B3C2D70115968C91811509F4AD
:1030300069C2033A22E5120708F022C3C801905280
:103040008115904208F423C3013E110509F45FC2C3
:10305000053E110518C3003E42E5140750F4003642
:1030600052E5150708F0A7CFC801925580349105A5
:1030700081CF980127573C472530310508F07BCF99
:103080000937BCE71B0709F04FC02091AC03309112
:10309000AD03232B79F18115A1F081E00E9457093E
:1030A0008091A4030E94900E89E0E5EAF3E0ABE58D
:1030B000B3E001900D928A95E1F78091AF03809380
:1030C0005A0386E0F701ABE5B3E001900D928A95D3
:1030D000E1F780915A038093B9038BE593E0F4DE26
:1030E0001092B903F7018581811104C08091A40376
:1030F0000E945A0F8091D9048770811561F0D70121
:1031000015968C91811539F08091900582FF03C04E
:1031100082E00E943A052C96E2E10C941534D70126
:1031200016968C91803126CF0A37FCE71F0709F0ED
:1031300042CF811509F4C5C0A090AC03B090AD0397
:103140002091A4032D832983BE016F5F7F4FC501AA
:103150000E9444082C0139813B87A4E6CA2EA3E0D3
:10316000DA2E01E010E022242A94D60117963C9032
:10317000179733FE53C06D907C90119712968D90E7
:103180009C90139746145704B9F41496BC91B987D0
:10319000232DF60146816B2F8B850E945E088115D9
:1031A00059F089850E946104281634F4D6011596D9
:1031B0009C918401192B282E48145904C9F431FE1E
:1031C00017C0F601F581F987232DD60116964C918B
:1031D0006F2F8B850E945E08811551F089850E94B2
:1031E000610428162CF4F60194818301192B282EF2
:1031F00030FE14C0FFEF2F1211C00130110571F421
:10320000232DD60116964C9160E08B850E945E08B6
:10321000811521F0F60185818401182BF8E0CF0E8D
:10322000D11C24EA33E02C153D0509F09ECF013076
:103230001105E1F58D8182958F703D81832B8F7013
:1032400011E0303108F410E01295107F182BA11412
:1032500040E2B40620F5A11451E0B50608F055C0CF
:103260000A2D812F8D704A2D811509F451C06AE015
:103270008FED97E00E946809282F30E02115310575
:1032800051F4402F6EE189EB97E00E946809282FE6
:1032900030E0811549F0F901F12B8F0107C0C5011C
:1032A00090528115904390F100E010E087E0E0EB50
:1032B000F3E0DF011D928A95E9F71093B8030093BC
:1032C000B7038091B7039091B803892B09F412CF0B
:1032D000F7018581811539F08FEF0E9457098091A0
:1032E000AF038093AE0386E0F701A0EBB3E001905B
:1032F0000D928A95E1F78091AE038093B90380EB3C
:1033000093E0E2DD1092B903F5CE1B29BB24A8CFD0
:1033100068E087ED97E0AECFC801975780389105F8
:1033200008F0DAC0003108F0E5CE64E670E080E035
:1033300090E06ADA8111DECE812C912C54010111CA
:1033400043C004E0AE014F5F5F4F6A01D601E02F3A
:103350001D92EA95E9F724013501FFEF4F1A5F0A44
:103360006F0A7F0AC501B4014FDA8983811509F418
:10337000C1CE813009F0ADC0A50194012E5F3F4F51
:103380004F4F5F4F2D833E834F835887C301B20158
:103390003BDA182F8A83811509F4ACCE8FEF810FA9
:1033A000833060F56D817E818F8198852DDA8B83E6
:1033B000811511F0C601D9DC2401350133E0430E3B
:1033C000511C611C711C17C0F5E68F169104A104F5
:1033D000B10409F48FCEC501B40116DA2FEF821AB9
:1033E000920AA20AB20A8111EFCF0150A8CF4D80F4
:1033F0005E806F80788453014201A8CF8BEF810FEC
:10340000833090F52401350143E0440E511C611CCA
:10341000711C6D817E818F819885F6D98B83811592
:1034200051F3C301B201F0D98C83811108C024018A
:10343000350154E0450E511C611C711CDCCF8B81A1
:103440009C818130AFEF9A0710F0982F88271630B3
:1034500029F0173031F00E94BE28E9CF0E946B2876
:10346000E6CF0E948C28E3CF143009F0C0CF6D81E5
:103470007E818F819885C8D9182F24013501B4E049
:103480004B0E511C611C711CC501B4016D5F7F4F57
:103490008F4F9F4FB9D9111509F42CCE811509F41E
:1034A00029CE8150990B4FEF489F9001499F300DD5
:1034B0001124E12FE150FF0B2E0F3F1F2150310946
:1034C00008F499CF8FE99FE00197F1F700C0000061
:1034D000F5CFC6014ADC8FCF0330A8E71A0709F4FD
:1034E00068C078F50130E8E71E0709F45AC00230D9
:1034F000F8E71F0709F48CC085E0011528E71207DB
:1035000009F450C0023AF2E51F0709F092CD21EE0E
:1035100030E02770332781E090E001C0880F2A95C2
:10352000EAF72091C8033091C503311509F4C3C0EF
:10353000F7013581311509F4B9C0282B2093C80350
:10354000D9CD043038E7130709F443C0053048E704
:10355000140709F473C00337BCE71B0799F6F7019A
:103560008581811509F4C6CD8091C503811509F4C3
:1035700077C00E94640FBECD223009F054CD209157
:10358000BE033091BF03232B09F44DCDFC01ED5A4E
:10359000FB4F20812E7F2083825B9B4F0E948D12E8
:1035A00042CD80E00E940A0884EC93E00E94090E5C
:1035B000A1CD8091C403883028F188508093C40342
:1035C00091E0883008F490E08091C40390FB80F98A
:1035D00013C09091C403892F86958695869598325D
:1035E00040F48F5F880F880F880F9770892B809326
:1035F000C4038091C40381608093C40384EC93E08E
:103600000E94090E8091C4038695869586950CC00C
:103610008091C40380FF0BC08E7F8093C40384EC31
:1036200093E00E94090E80E00E94780763CD8160DC
:103630008093C403813011F789E0DECF8091C40309
:103640008695869586958F5F8F71863008F080E02D
:10365000880F880F880F9091C4039770892BAECF85
:103660001092D6040E9463050E94440A88579C4E1B
:103670009093C7038093C60381E08093C5033ACD3E
:10368000023B42E5140741F525EE30E042CFD70179
:1036900016968C91803100F5812F99278F7199278B
:1036A0008230910509F433CF4297EDCF8095822384
:1036B0008093C8031FCD322F3823311569F0982F1E
:1036C000909592239093C8030E945B05D7011596AD
:1036D0008C91811509F40ECD8091C503811509F4F3
:1036E00067C0C090D604D090D5040E94440A885781
:1036F0009C4E9093C7038093C603F7018581811583
:1037000009F456C08D2D8C298D79811184C0011545
:10371000F0E51F0700F5011520E4120708F082C04C
:10372000063E110509F444C0C8019052811590422B
:1037300008F07FC0D70116968C91803108F463C0E1
:10374000C80199271092D8048D329105E9F482E0DE
:103750008093D80472C0003EB2E51B0708F046C053
:10376000003CE2E51E0720F5003AF2E51F07E0F411
:10377000003622E51207E0F4C80192558034910525
:10378000B8F01092D804C8018E32910508F062C0DA
:103790008832910508F04FC08E31910508F04DC078
:1037A00004974A97A0F237C0043B32E5130749F764
:1037B000F7013580311409F457C00E35FCE71F07B7
:1037C00009F44EC00F352CE7120751F00D353CE7D8
:1037D000130709F049C080911001811509F440C018
:1037E0001092100180E00E94B21284CC09374CE79D
:1037F000140728F407375CE71507D0F6C2CF0B375C
:103800008CE71807D4CF812F8F71843189F28631EC
:1038100011F41092D8040E94640F8091C8030E9492
:103820005505C6CFD70116968C91803108F088CF08
:10383000BFCFC80187CF8A9771F78091C8038115E0
:1038400031F08091D80492E089278093D8040E94B7
:10385000360EAECF8C34910581F38D329240ECCF91
:1038600081E08093100146CC80911001811169C0E4
:10387000C80197558115914008F0FFC05801F8EF35
:10388000AF22BB24A114B10409F034CCF801FF2706
:1038900054E0EE0FFF1F5A95E1F79F01225B3B4F6B
:1038A0006901D70115968C91ED5AFB4F908180FBF1
:1038B00090F99083811509F4D9C10E94440A90932C
:1038C000D1048093D004F60182818F5F828380913E
:1038D000D8049091D604892B83838091D504848366
:1038E0004681578166857785C6010E947D09D6018C
:1038F00015968C9181FF5801B092CF04A092CE040E
:10390000D70115969C91911509F42EC61092D204F8
:10391000980130572332310508F011C684E090E059
:103920000E9465349093900580938F05F801E150D3
:10393000F047E232F10508F0E2C1E353FB4C0C948E
:10394000C333380150EE651A71085090D704809146
:10395000D604582A8091D504582A88E06816710444
:1039600008F05EC098012770332781E090E001C025
:10397000880F2A95EAF7311409F44FC0582AD70165
:103980008D919C910E94DD0421E030E0F90102C09C
:10399000EE0FFF1F8A95E2F7FA87E987209144042A
:1039A000309145043E832D8340914C0450914D0449
:1039B0005C874B876BECC62E63E0D62EA12CB12C16
:1039C000511005C0D60112968C9181111BC0F601D1
:1039D000838190E029853A8582239323892B91F076
:1039E0008085982F9770911101C087E038E06316A9
:1039F000710408F066C0311409F45FC086958170C7
:103A0000811164C09FEFA91AB90AAFE0CA0ED11C98
:103A1000B8E0AB16B104A1F61CC080955822AFCF18
:103A2000311038C080914C0490914D04081719074B
:103A300081F410924D0410924C041092480410929C
:103A4000490410924A0410924B04109247041092B9
:103A500046048091440490914504009709F408CFEE
:103A6000E8E06E16710408F0EBC0652D0E94BC08FA
:103A7000811103C081E00E94B212F7018581F80133
:103A8000E851FC47E730F10508F03ACFE151FB4C33
:103A90000C94C33310934D0400934C040E949B0B71
:103AA000609348047093490480934A0490934B04B4
:103AB000109247041092460462CF82FB882780F957
:103AC0009FCF311409F49ECF80FF9CCFD6018D90FB
:103AD0009C900815190519F4311409F493CFED8160
:103AE000FE81EC15FD0509F48DCFD6011D96ED91F3
:103AF000FC91309721F08081811509F483CF652DE9
:103B0000C6010E94BC08811509F47CCF81E008152C
:103B1000190509F080E0482E43208114910441F0FA
:103B2000411006C0EB85FC858E169F0609F06ACF12
:103B300080E00E94B212D0924504C092440481E019
:103B4000809343048FE08A9DF0018B9DF00D11243A
:103B5000E553FC4F85818093CA0341100EC0811448
:103B6000910459F0808191819C0124503109213ABE
:103B7000310508F049C00E94150A8FE08A9DF001C6
:103B80008B9DF00D1124E553FC4FC680D780C601F4
:103B90009A9581159F4110F420EED2229924939496
:103BA000C60101978F339E4708F0912C8FE08A9DC4
:103BB000D0018B9DB00D1124A553BC4F1996ED91EA
:103BC000FC911A97309731F01B966D917C9181E0B2
:103BD000099598229114A9F08FE08A9DF0018B9DA0
:103BE000F00D1124E553FC4F868197810E942E042D
:103BF0008093C903C60148E06416710440F40E9432
:103C0000A70B0E94360E0AC00E94130FB6CF04976E
:103C1000813A910548F48C2D0E94E109411409F480
:103C200027CE0E94360E66CA0E94360E8FE39CE9AC
:103C30000197F1F700C000008C2D0E94990EEECF85
:103C4000DC012D913C910217130741F4311009C09A
:103C50001092430480E00E94B2120ACE311409F49B
:103C600007CEFC01808585FD03CEF4CFF9014485A4
:103C7000558566857785C9010E947D09D60115960F
:103C80008C9181FF3DCEC6010E9471128091CE04BD
:103C90009091CF040817190709F032CE1092CF0483
:103CA0001092CE042DCE06E221EE41EE6AE17CE7D1
:103CB0000E94F6151FCA07E225EE45EE6BE17CE790
:103CC000F7CF06E221EE40EE68E17CE7F1CF07E2B4
:103CD00025EE44EE69E17CE7EBCF06E221EE42EE11
:103CE0006CE17CE7E5CF07E225EE46EE6DE17CE78F
:103CF000DFCF08E221E045EE6EE17CE7D9CF80918D
:103D00008F05816080938F0560918F05709190057C
:103D100084E090E00E9493340E946D0FEBC9809183
:103D20009005886080939005EFCF80918F05826029
:103D3000E9CF80918F058460E5CF80918F05886001
:103D4000E1CF809190058160EDCF809190058260F8
:103D5000E9CF80918F058061D5CF80918F058062FA
:103D6000D1CF80918F058064CDCF0E946D0F80915F
:103D70008F058068C7CF80918F058C60C3CF8091FD
:103D800090058360CFCF80918F058E7FBBCF8091D0
:103D90009005877FC7CF80918F058D7FB3CF8091AE
:103DA0008F058B7FAFCF80918F05877FABCF8091C1
:103DB00090058E7FB7CF809190058D7FB3CF809196
:103DC0008F058F7E9FCF80918F058F7D9BCF8091B8
:103DD0008F058F7B97CF0E946D0F80918F058F7716
:103DE00091CF80918F05837F8DCF809190058C7FBF
:103DF00099CF80918F05992782FF939590FB82F947
:103E000090FB83F97FCF80919005982F909590FB40
:103E100080F990FB81F986CF90918F05892F8F7B58
:103E200096FF80646FCF0E946D0F90918F05892F50
:103E300097FB87F9805866CF61E08EE090E00E94A2
:103E4000793462CF60E0F9CF90918F05892F8F7E12
:103E500094FF806157CF90918F05892F8E7F90FFBF
:103E6000816050CF90919005892F877F93FF886064
:103E700059CF89E276C389E282C30737BCE71B07C3
:103E8000F9F00837ECE71E0731F19801205E324562
:103E90002032310528F5911123C00F7181E090E0A7
:103EA0009C0102C0220F331F0A95E2F78901622F9D
:103EB00083E090E00E947934802F0E9489041AC91F
:103EC00081E0911551F00E948F0443E062E081E0AF
:103ED0000E9411050FC982E0F4CF0E949904F5CF2A
:103EE0004091D40480918E05282F30E020953095A4
:103EF00070E024233723232B19F048234093D40464
:103F00000B373CE7130741F4911509F4F3C80E94FD
:103F100064040E94DD08EEC8003442E5140708F08E
:103F200055C0003252E5150708F057C0011580E56D
:103F3000180750F50115A0E41A0708F064C09115A0
:103F400009F479C00A35FCE71F0709F4CDC008F071
:103F5000B2C001303CE7130709F4C4C003304CE79A
:103F6000140709F4B9C001151C4709F064C00E9488
:103F70006D0FAFEFB4E3ECE0A150B040E040E1F7EB
:103F800000C000000E94670D980130552115324095
:103F9000B0F6980145E0369527954A95E1F7822FCE
:103FA0008F702091D40430E041E050E0082E02C030
:103FB000440F551F0A94E2F724233523232B09F4D9
:103FC000BECF9111A6CF1092D6042BCE9801205CC3
:103FD00032452032310508F0B2CF802F8F71209109
:103FE000D40430E041E050E0082E02C0440F551FD9
:103FF0000A94E2F724233523232B09F4A0CF91154B
:1040000009F478C886CFF7018681803108F097CF10
:10401000911111C0212F2F7081E090E002C0880F14
:10402000991F2A95E2F72091D40430E0822393234C
:10403000892B09F05FC8F70187819085009709F403
:1040400057C00E9461068C01F701B580A680A2943A
:104050002FE0A2228091D9048770811501F1CB2C29
:10406000B114F1F0812F807F803461F080E2800F05
:104070008830A8F0812F807E803221F4023078F0E1
:10408000A11469F08091900582FF09C082E00E942E
:104090003A058091D9048770CC24C3948111C12C36
:1040A000E12FE295EF70103C08F094C0F0E0EA5088
:1040B000FB4C0C94C3330B358CE71807B9F0809197
:1040C0009005002482FF0394802D0C351C4709F0D5
:1040D000B2CF0E94F20DAFCF6FEF7FEF80E090E0A4
:1040E0000E9493340E94990F81E0F3CF80E0F1CFDA
:1040F0008581C080D180811569F0C6010E94791345
:10410000182F682FC6010E94A704B601812F0E94B4
:104110005E1397CFC6010E94DD04182FF6CFF12F52
:10412000FF70DF2E103118F0D29490EFD922B11425
:10413000A9F0D11459F080E2800F883010F00111FD
:1041400007C08D2D0E9455050E94360E802F40C05D
:104150008091D8048D298093D804F6CF802F0E94B7
:10416000130FD114B9F180E2800F883010F00111E3
:1041700004C08D2D0E945B0506C0D0948091D804A8
:104180008D218093D8040E94360E24C0212F2F70D9
:10419000D22E107F103219F0D29480EFD822011560
:1041A00049F0013009F483C0B11409F48FC0A1149F
:1041B000A9F1CCCF8091900582FD2CC0B11421F1E2
:1041C000D11429F08D2D0E9455050E94360E80E0F5
:1041D0000E94990EC11409F4DBC08091D90480FDBE
:1041E000D7C0D70115961C928695869586950E9414
:1041F0008F04C7010E9464178091D9048695869523
:1042000086950E949904C4C080E00E94130FD114C7
:1042100009F3AFCFB11469F1A11004C08D2D0E9434
:104220008A0ED8CF31E0A31210C01091D5048D2D85
:104230008123D81679F20E94440A9093DD0480937A
:10424000DC041D291093D504C5CF45E0A412C2CFCC
:104250008D2D0E948A0E8D2D0E94A20A8091D70476
:104260009D2D9823D91609F4B5CF8D298093D704B5
:10427000B1CFA11012C08D2D0E94540F8D2D0E9420
:10428000A20A8091D7049D2D9823911509F4A2CFFD
:10429000D094D822D092D7049DCF51E0A5129ACFC6
:1042A0008091D6048D21811509F494CFE4CFB11407
:1042B00029F086E0A81608F08DCFB0CF95E0A916BA
:1042C00008F088CF8D2D0E94540F84CFA114D1F314
:1042D000093349F4AFEFB7EEE3E0A150B040E0405E
:1042E000E1F700C00000802F0E94130F73CF812FD1
:1042F000869586958370811561F0813009F06ACFCB
:10430000C8019370B11002C080E090E00E94B9092A
:1043100061CFC8019370B11002C080E090E00E94AC
:10432000910958CF6B2D802F0E94E00A53CF812F27
:10433000837081113BC0B11027C0402F4295469534
:104340004770440F440F802F8F70042E01C0880FD8
:104350000A94EAF7202F207104FF07C02FE030E015
:1043600001C0220F4A95EAF720951695169513700D
:104370001230B9F0133099F030918D05113071F091
:10438000822B83230E9489040E9482090E94770461
:1043900060E0C7010E94A3130C948B18832B822B1F
:1043A000F1CF822B90918D058927ECCFB11451F17B
:1043B00010FFEACF402F429546954770440F440FB7
:1043C000802F8F70042E01C0880F0A94EAF7202FE7
:1043D000207104FF07C02FE030E001C0220F4A9592
:1043E000EAF72095169516951370123091F0133058
:1043F00071F030918E05113049F0822B83230E9499
:104400008C04C2CF823008F4BFCFD4CF832B822B51
:10441000F6CF822B90918E058927F1CF1F70B114B2
:1044200039F0812F0E948F04802F0E948A0EACCF1A
:10443000802F0E94540F812F0E949904A5CF023F24
:1044400071F170F4003FC9F0013F91F0B11409F42B
:1044500065C0A11409F45FC0802F0E94990E94CF0B
:10446000033F21F1043F91F78091900582FD2AC01E
:10447000812F8F71B11401F316C0B11469F0F5E00A
:10448000AF1608F081CF1F7181E090E0012E01C0CE
:10449000880F0A94EAF7BECF26E0A216F2CF812F4A
:1044A0008F71B110C9CF0E948F046ECF80E0B1141C
:1044B00009F4A5CF1F7181E0012E01C0880F0A9475
:1044C000EAF79DCFB114C1F08091D9048770843090
:1044D00049F41092D9041092DB041092DA04812F6F
:1044E0008F71AACF35E063E0A31608F04DCF812F7E
:1044F0008F710E948E0A48CF45E0A41640F01092BA
:10450000D9041092DB041092DA0464E0F0CF81E069
:104510000E943A0539CF812F8F71C5CFA114F9F2CE
:10452000093349F45FEF87EE93E0515080409040AB
:10453000E1F700C00000802F0E94130F25CF063145
:10454000FCE71F0709F099CC8091D6048A7A91E0A4
:10455000811101C090E09093D304811509F489CCB6
:1045600085E30E94E1095DCB06312CE7120709F0D3
:1045700084CC8091D304811509F47DCC85E30E941D
:10458000150A4FCBA0E0B0E0E8ECF2E20C94043462
:1045900080912703803108F049C08091260381155E
:1045A00009F444C0C091D80289E0D82E8091D70286
:1045B0008C17E1F1EC2EF12CDC9EE0011124FE01C0
:1045C000E752FD4F84818115B1F1918180912203E1
:1045D000981331C090818091210398132CC085815C
:1045E000811129C0028113818091230390912403BA
:1045F000081B190B60E081E293E00E94A3130E9464
:10460000DB1508171907B8F4809127038F708061B4
:1046100080932703C152DD4F88818F70806188832A
:1046200081E293E00E9464170E943005CDB7DEB7A7
:10463000E7E00C942034E7012196C770B7CFAFE0D4
:10464000B0E0E5E2F3E20C94FC338C0186E0F80183
:10465000DE011A9601900D928A95E1F7F801F58036
:10466000E48081E2882E83E0982E809125038111D9
:1046700017C0E11491F0F11409F480C1C8010E943F
:10468000D213811509F47AC189E0F801A1E2B3E0FF
:1046900001900D928A95E1F775DFFF24F3946AC0CB
:1046A000A280B380D09026038091230390912403AD
:1046B0003501681A790AD11409F411C1C0805180FA
:1046C00060E081E293E00E94A3130E94DB1568166C
:1046D000790608F0B6C0E11401F380912203F801D5
:1046E0009181E0902703F0E1EF1608F064C0981381
:1046F00020C090912103F801808198131AC0209165
:10470000280330912903878190852817390789F478
:10471000F1104BC08E2D8F7080618093270381E252
:1047200093E00E94641780912703F8018683F12C9F
:1047300021C0F1103AC040E0652D8C2D0E94480D3B
:1047400040E0652D8C2D0E94480DF82E8111EFCF91
:104750008A859B850E94C513292F22952F7090343E
:1047600070F49F702230A0F09115B1F0F80196819D
:10477000903190F48F2D2F96EFE00C9418342A5F2F
:104780002F70223068F0C8010E946417FD2CF2CF10
:10479000911511F0811571F3805E883058F3F3CFD5
:1047A000803F40F3815F8330F9CF809127038160A0
:1047B00080932703BCCF98131EC090912103F8016A
:1047C0008081981318C02091280330912903878194
:1047D00090852817390779F4F1100DC0E682C801D9
:1047E0000E94641789E0F801A1E2B3E001900D9204
:1047F0008A95E1F752CFC8010E94D213811509F4BE
:10480000BDC0F11409F4BAC080912703803208F4C6
:104810003BCF80912103909122039A838983BC82AC
:10482000AB82809125038D831E82EF8280912803C5
:104830009091290399878887CE0101960E94641779
:1048400023CFD0902703F0E1DF1650F481E293E00C
:104850000E94641789E0F40111928A95E9F767CF05
:10486000E11409F41ACF90912203F8018181981381
:104870001AC0909121038081981315C020912803BC
:1048800030912903878190852817390761F4F11049
:104890000AC0D682C8010E94641789E0F40111920F
:1048A0008A95E9F7FACEC8010E94D213811509F45E
:1048B00065C0F11409F462C080912703803208F4C6
:1048C000E3CE80912103909122039A838983BC8255
:1048D000AB82809125038D831E82DF82A7CF60E0AB
:1048E00081E293E00E94A3130E94DB15681679060B
:1048F00008F0B0CFE11409F4D0CEF11409F43EC0B1
:1049000090912203F801818198132EC09091210388
:104910008081981329C02091280330912903878131
:1049200090852817390701F580912303909124037E
:10493000A81AB90AF8ECAF16B10408F053CF809169
:10494000270380FD4FCF803108F44CCFF8018683D8
:10495000982F907F903F09F442CF982F907F905FDF
:104960008F70892B86833BCFC8010E94D21381119F
:104970008BCE80912703816080932703C8010E941A
:1049800064178BCEA2E1B0E0E8ECF4E20C940734BB
:104990000A871B872C873D874E875F87688B798BBB
:1049A0008A8BCE010A964BDE811128C02091D70256
:1049B0003091D80289E0FE013A96DE01119601900D
:1049C0000D928A95E1F78E858115C1F0822F90E0D6
:1049D00001968770992738171906D9F099E0929FA8
:1049E000D0011124A752BD4FFE01319601900D92C6
:1049F0009A95E1F78093D7020E94300519E08091E3
:104A0000D8029091D702891312C06296E4E00C9408
:104A100023340E946D0F1092D7021092D80289E0C1
:104A2000E1E2F3E0DF011D928A95E9F7E7CF189FF5
:104A3000C001112487529D4F02DE811531F3809110
:104A4000D80290E00196877099278093D802D7CF3B
:104A5000EF92FF920F931F93CF93DF9380918A057C
:104A6000E091F401CDE0811130C0CDB7DEB7E6E0D2
:104A70000C942134D1E0DE0FD093F401EE2EF12C12
:104A8000CE9FF0011124EE5DFA4F84818115E1F093
:104A900087819085892B21F481859285019651F437
:104AA0000081118122813381448155816681778122
:104AB000808568DFCE9DF001CF9DF00D1124EE5D65
:104AC000FA4F14821092D804ED2F80918A05E817CE
:104AD00088F210928A051092F401C7CFA4E0B0E0EA
:104AE000E4E7F5E20C94FA3320912105298397E05D
:104AF000992E01E010E02DE0322E34E0532E882470
:104B00008394809120059981891307C0A1DF0E94B9
:104B10007F082496E1E10C9416349981892F90E066
:104B20009C838B83FC01EE0FFF1FEA5EFA4F8081AE
:104B30009181989ED001999EB00D1124FD01E25201
:104B4000FB4FFA83E983248121115BC060908A05C1
:104B5000E2E2F5E060E070E0712C661508F04FC00D
:104B6000A384B484A981BA81CD90DC902FEF3FEF6C
:104B7000412C442D50E07601E40CF11CE40CF11CB6
:104B8000D701ED90FC90E114F10439F0AE14BF04AC
:104B900009F0A90143949A01ECCF2F3F3207D1F1DC
:104BA000D80102C0AA0FBB1F2A95E2F77A2A980102
:104BB000042C02C0220F331F0A94E2F7A9014150CE
:104BC00051097416150629F5369EF001379EF00D31
:104BD0001124EE5DFA4F989ED001999EB00D1124DC
:104BE000A252BB4F12962D913C9113973087278389
:104BF0005482108211829287818715968C920E942E
:104C000090088B819C8101969A8389838370898324
:104C100078CF14826F5F7F4F3D969FCF10928C05A7
:104C200010928B051092110180912005809321052F
:104C30000E947F080DCFACE1B0E0E1E2F6E20C9417
:104C4000F9334B8B5C8B6D8B7E8B8F8BB92E988F52
:104C5000A92E91111092D804188A198A1A8A86E00E
:104C6000FE017396DE011A9601900D928A95E1F786
:104C70005F888091900582FF1FC00E94440A2091A6
:104C8000DA043091DB04821B930B8838934138F0AF
:104C90008091D90482FD03C082E00E943A050E94FF
:104CA000440A2091DC043091DD04821B930B883888
:104CB000934110F00E9463055114D9F05E86BF86BF
:104CC00061E0CE010A960E94A31361E0CE010A962C
:104CD0000E94A31361E0CE010A960E94A3134C0127
:104CE00080356CE7960791F4A11419F181E0809367
:104CF00011015E86BF860A851B852C853D85452D65
:104D00005B2D688979898A893DDECDC081359C47D4
:104D100021F4A11471F082DFECCF82E588168CE7D4
:104D2000980639F4A11429F0809111018111F3CF73
:104D3000DDCF4EEDE42E44E0F42E412C612C712C9D
:104D4000D7016D917C91CC24CA94DD24DA9480E063
:104D5000282F30E0FB01E80FF11DE80FF11D408125
:104D600051814115510539F08416950609F09601D7
:104D70008F5F6901EDCF10E0BFEFCB16DB0609F4C2
:104D80004EC0F701448110911101411110E0D7018B
:104D900015963C90159716969C911697A11409F4B8
:104DA00005C1111509F402C1311017C021E030E02E
:104DB0000C2C01C0220F0A94EAF7922B16969C93B2
:104DC00020911E0530911F052233310530F422E376
:104DD00030E030931F0520931E05E1E0F0E002C0B3
:104DE000EE0FFF1F8A95E2F7CF010197D7011696C4
:104DF0002C912817190699F4C0908B05D0908C053A
:104E0000C114D10409F453C00E94440A8C199D09AD
:104E1000C39708F44CC081E0F701848311E0412A74
:104E2000BFEF6B1A7B0AE7E0EE0EF11CF8E06F169D
:104E3000710409F085CFA11409F417C1411409F4D4
:104E400014C10E94440A90938C0580938B05809135
:104E50008A05883040F591E0980F90938A0599E093
:104E6000FE013A96DE01119601900D929A95E1F7B6
:104E70005D82BE822DE0829FC00111248E5D9A4F1B
:104E800029E0FE013196DC0101900D922A95E1F7AF
:104E90002FEF3FEFDC011A963C932E9319971C9647
:104EA0009C928E921B976C96E2E10C9415342091A3
:104EB000210580912005922FE0E0F0E001E0281725
:104EC00009F448C0422F50E0FA01EE0FFF1FEA5EDE
:104ED000FA4F2080318037E0329DF001339DF00D94
:104EE0001124E252FB4F608171817C8F6B8FB0E0A7
:104EF00030E0A0E0EB8DFC8DEA0FF11DEA0FF11D13
:104F0000C080D180C114D104E1F0F7010190F0819B
:104F1000E02DFA8FE98F30E007C0E1E0C616D70632
:104F200009F0E0E0BE2B3F5FE98DFA8DE30FF11D44
:104F3000E30FF11D608171816115710571F7AF5F3C
:104F4000D9CFB11581F13A17C8F4E1E0D701149631
:104F5000EC93F70190932105EE15FF0509F45FCF5F
:104F600090E0FC01EE0FFF1FEA5EFA4F7182608253
:104F70000196837099278093200551CF37E0329DA9
:104F8000F001339DF00D1124E252FB4F0483EE1526
:104F9000FF05F9F2291302C09F5F93709A012F5FFA
:104FA0003F4F23708CCFE0E0F0E0F8CF292F30E0C6
:104FB000311024C061E070E002C0660F771F8A954F
:104FC000E2F7CB0101972817390791F010E0E1E0F3
:104FD000F0E002C0EE0FFF1FCA94E2F76F01C09429
:104FE000D70116968C9116978C2116968C9317CF15
:104FF000411569F3C3010E949008E8CFA9010C2C68
:1050000002C0559547950A94E2F7C901019782239A
:105010009323892B39F540FF25C0D70112968D9136
:105020009C91892BD1F087E0FE013196DF011D9222
:105030008A95E9F70E94440A9C018B839C8384E053
:105040008D83F70192818381792F988789870981E0
:105050001A8144E05E816F8195DCD70115961C9220
:10506000132DB5CF142F1170B2CF909121058091DF
:105070002005981731F032DDB1E04B1609F413CF5B
:1050800038CEE6DC10928C0510928B050E947F08CA
:10509000F3CFA6E0B0E0EFE4F8E20C9407340E940E
:1050A000440A8C018091AB029091AC028017910769
:1050B00071F019821A820E94440ABC0149815A8106
:1050C00080E090E0B8DD1093AC020093AB0226962E
:1050D000E4E00C942334A6E0B0E0E1E7F8E20C94BD
:1050E00009349093A8028093A702811520E29207C9
:1050F00030F40E94FE0E2696E2E00C94253480EFF8
:1051000089838A830E94440A8160BC0149815A8153
:1051100081E091E090DDEFCFA6E0B0E0E2E9F8E2D7
:105120000C9407348C019093A8028093A702011578
:1051300080E21807B0F4802F0E94130FC801805E30
:105140009109089728F06AE57FE00115110511F42F
:1051500064E57FE0C8010E9458042696E4E00C94C0
:10516000233480EF89838A830E94440A8160BC01D2
:1051700049815A8181E090E05EDDEFCFCF93DF93EC
:10518000D82FC92FA8DF8D2F9C2FC6DFDF91CF919D
:1051900008950F931F93CF93DF938C01862F6AEBB3
:1051A00073E00E94C615892B91F4C091BA03D09187
:1051B000BB03209761F0F8018281833039F4CE017E
:1051C000DDDFCE01DBDFCE01D9DF01C0E0F7DF910B
:1051D000CF911F910F9108950F931F93CF93DF935A
:1051E0008C01EB016AEB73E08C2F0E94C615892BB2
:1051F00009F057C0FE01FF27D80112968C91129733
:10520000EA5BFD4F8130A9F415968C9182FD4EC06A
:1052100080FF4CC082E080838091BC039091BD03ED
:105220000097B9F48091BA039091BB030097C9F13C
:1052300010C08230A1F515968C9182FD26C080FDAC
:105240000AC083E080838091BE039091BF030097E2
:10525000F1F041DF26C084E080838091C00390910B
:10526000C1030097B1F78091BA039091BB030097F7
:1052700001F184DF8091BC039091BD03009749F751
:105280008091BA039091BB03E4CF85E08083809145
:10529000BA039091BB03009721F070DFF1CF86E055
:1052A0008083DF91CF911F910F91089581E08083DA
:1052B000B9CF8091BC039091BD03B8CF0F931F93DA
:1052C000CF93DF938C01EB016AEB73E08C2F0E948C
:1052D000C615892B71F4DD27CA5BDD4F8881F80183
:1052E000128218828330E9F048F4813059F082301C
:1052F00081F0DF91CF911F910F9108958430B1F02B
:105300008530B9F78091BA039091BB03009789F378
:1053100006C08091BC039091BD03009799F3FCDE19
:10532000E8CF8091BE039091BF03F7CF8091C00377
:105330009091C103009799F72091BA033091BB0374
:105340008091BC039091BD0321153105F9F20097BE
:1053500031F7C901E4CFA6E1B0E0E1EBF9E20C944A
:10536000FD33FE01319686E1DF011D928A95E9F752
:105370000AE211E093E3C92E91E0D92EEE24E394E2
:10538000F12C9E2E8F2EAA24A394B12CF80181918A
:105390008F018F3F09F44BC0F894E82FE295EF702E
:1053A000F0E021A18F70A50102C0440F551F8A951E
:1053B000E2F7CA01922F982B91A392A1809589239D
:1053C00082A3789400C0A3E3B1E0692C782C970104
:1053D000209530956D91F301819191913F016F3F3F
:1053E00009F44BC0462F42954F70405E50E0FA01E1
:1053F000408150E06F7002C0559547956A95E2F77D
:1054000040FD3BC08E299F29A30142505109FA015A
:1054100091838083F1E0AE33BF07E1F6F80182911A
:105420008F3F11F00E945F0740EA4A95F1F7EE0CBA
:10543000FF1CC016D10609F0A9CF46E150E0692D46
:10544000782D8EE492E00E943934892BC9F086E1F0
:10545000E92DF82DAEE4B2E001900D928A95E1F7C6
:1054600081E08093D6010E94440A9093D5018093F5
:10547000D4016696EEE00C94193482239323C4CFB2
:105480008091D6018115A9F30091D4011091D50125
:105490000E94440A801B910B059758F346E150E0A7
:1054A0006EE472E08EE892E00E943934892B49F074
:1054B00086E1EEE4F2E0AEE8B2E001900D928A956A
:1054C000E1F71092D601D5CFCDB7DEB7AC970FB6C6
:1054D000F894DEBF0FBECDBF85B7806885BF85B7A6
:1054E000806885BF84B7877F84BF0FB6F894A8957E
:1054F00080916000886180936000109260000FBE10
:1055000080E890E00FB6F89480936100909361007A
:105510000FBE81E080930F018DE597E09093AB0182
:105520008093AA010E942C080E94C3140E940715B0
:105530000E9486150E94910C0E94EE0C8091E20060
:1055400084608093E20078948091A602811599F09E
:105550008091E9001091EC008F7017951127179535
:10556000182B1092E9008091E80083FD0E94AE0F95
:105570001F701093E90082E084BD93E095BD9AEF1F
:1055800097BD80936E000E941414811102C00E9486
:1055900090160AE211E0D8018D918D018F3F11F034
:1055A0000E945F07B1E003331B07A9F703E311E093
:1055B000F80181918F018F3F11F00E945F07F1E0A8
:1055C0000E331F07A9F786E1EEE8F2E0DF01282F8E
:1055D0001D922A95E9F7EEE4F2E0DF011D928A952B
:1055E000E9F780E090E00E946534833E9E4F21F40D
:1055F0000E94141481112EC063EE7EEF80E090E0D3
:105600000E94933460E082E090E00E94793481E06F
:1056100080938D0561E083E090E00E94793460E042
:1056200074E184E090E00E9493341982CE010196E7
:105630000E94090E0E94901640E050E0BA018FE0EF
:1056400090E00E948B3440E050E0BA0183E190E0AA
:105650000E948B3482E090E00E945D348093660269
:1056600084E090E00E9465349093900580938F05CC
:1056700072DEEFEFF6E721E0E150F0402040E1F785
:1056800000C0000068DE80918E0280FF08C06FEFCE
:105690007FEF80E090E00E9493340E94670D83E0EA
:1056A00090E00E945D340E948904259A2D9A3E9ACA
:1056B000469A3F9A479A269A2E9882E280938000D3
:1056C00089E1809381008FEF9FEF90938700809313
:1056D00086000E940D130E940D1380E091E09093CC
:1056E000CE028093CD028091A602853069F480912C
:1056F000A602853009F45EC00E946D0F0E940D1352
:105700000E9482090E94770426DEE7E6AE2EE2E0E0
:10571000BE2E0EE812E0D801F501219131918D9154
:105720009D9142E0ED37F40709F480C0281739074E
:10573000A1F37EE8872E72E0972E512CD401ED90D4
:10574000FD904D01F501619071905F016E147F0431
:1057500051F16E247F24412CCC24C394D12CC6015A
:1057600086219721892BB1F049825A820E94440AEE
:105770009C838B83F1E0FD8391E096012E213F21F4
:10578000232B09F490E09E8349815A816B817C81AF
:105790008D8151DA4394CC0CDD1C29E04212DFCF1D
:1057A000F501F292E29253943BE05312C7CF0E946C
:1057B0009B0B41C08091A602843051F180E00E9491
:1057C0000A0880E00E9477041092640288E190E069
:1057D000A0E40FB6F894A895809360000FBEA09344
:1057E000600083B7817F846083BF83B7816083BF9C
:1057F0007894889583B78E7F83BF0FB6F894A89569
:1058000080916000886180936000109260000FBEFC
:10581000A2DDEEE8F2E081919191892B09F0C0C5FB
:1058200024EA32E02E173F07B1F761CF2817390776
:1058300009F07FCF2EDCE0904604F0904704E1149D
:10584000F10491F18090810290908202A0908302F5
:10585000B09084020E949B0B681979098A099B0900
:1058600080907D0290907E02A0907F02B090800296
:10587000681579058A059B05B8F0C7010E94FE0EE0
:1058800010924704109246041092810210928202F4
:10589000109283021092840210927D0210927E0276
:1058A00010927F0210928002C090CE04D090CF045C
:1058B000C114D10439F1A090D004B090D1040E9459
:1058C000440A7C01EA18FB08C6010E94DB158E150C
:1058D0009F05C0F42091CE043091CF04C9019927CF
:1058E000287F3327232B09F059C144E0880F991FE3
:1058F0004A95E1F7825B9B4FDC0115962C9122FFC4
:105900000E948D1280911101811511F1E0908B059B
:10591000F0908C05E114F104D9F00E94440A8E192C
:105920009F0920911E0530911F052817390780F423
:105930009091210580912005981709F432C1CED8A5
:1059400010921F0510921E0510928C0510928B0567
:105950008091C503811569F00E94440A2091C60315
:105960003091C703821B930B8F3F9F4710F40E9417
:10597000640F86E0E4E5F3E0DE01119601900D92FC
:105980008A95E1F790905503B0905603F090570335
:10599000A0905803E09059031092560310925703B9
:1059A00010925803109259038F2D8B29811509F4F9
:1059B00041C0C0908702D09088020E94440A9C0196
:1059C0002C193D0990915203911509F4E4C4253135
:1059D000310580F19F3F19F09F5F90935203B114FE
:1059E00059F00E94120991E01B140CF09FEF899F5F
:1059F000802D112480935603F11459F00E9412094E
:105A000091E01F140CF09FEF899F802D112480934B
:105A1000570380915603811569F0D0905703D11434
:105A200049F00E940409809356038D2D0E940409B9
:105A3000809357038A2D8E29811509F441C0C090A7
:105A40008502D09086020E94440A9C012C193D09CF
:105A500090915103911509F499C42135310580F1D4
:105A60009F3F19F09F5F90935103A11459F00E943A
:105A7000320991E01A140CF09FEF899F802D1124B8
:105A800080935803E11459F00E94320991E01E14EA
:105A90000CF09FEF899F802D1124809359038091F2
:105AA0005803811569F0D0905903D11449F00E9430
:105AB0000409809358038D2D0E9404098093590393
:105AC00080915503981219C080915603811511F0E9
:105AD0008B1113C020915703211511F02F110DC008
:105AE00090915903911511F09E1107C03091580300
:105AF000311103C0822B892B81110E94B70A86E0E5
:105B0000FE013196A4E5B3E001900D928A95E1F78C
:105B10000E948209F82E80918902F81639F0F092DD
:105B200089020E949B0B8F2D0E9477048091A60210
:105B3000843009F0D8CD83E08093E9008091E800BB
:105B400082FFD1CD8091E80090E085FF05C00E94E2
:105B5000600C811579F191E08091E8008B7780935A
:105B6000E800911509F4BFCDE090A902F090AA02D7
:105B7000E981E114F104E1F1EE3F09F05CC08A81B2
:105B8000833020F08550833008F055C0EA81EE3034
:105B900008F051C0F0E0EE5FFA4CF5C580E090E00F
:105BA000ABCE0E94282510928C0510928B050E9486
:105BB0007F08CECE30E2C32ED12CFE0131967F017C
:105BC0008091E80085FD0AC08091E8008B77809382
:105BD000E8000E94600C811599F3BDCF8091F1001F
:105BE000D7018D937D01B1E0CB1AD10849F7B3CF2E
:105BF000E43148F4E11551F0E150E33138F4F0E0DC
:105C0000E05FFA4CC0C5EE3F09F4C0CF8FEF898347
:105C100012C01A8289E08B830EC08A81823081F0A3
:105C20008330B1F0813091F70E949B0BC2D56B831A
:105C30007C838D839E83CE0101960E94B00C53CD50
:105C400088E290E03AD61B821C821D828E83F3CFBD
:105C50008091A4029091A502892B69F3FE013196EF
:105C6000D8018C9111969C910E5F1F4F9283838374
:105C70003296B2E0043A1B0799F7DDCF8A81823071
:105C800029F66B817C818D819E8193D588E290E09D
:105C900030D6D1CF4C816B818A810E942F139827F7
:105CA000892798279E838D83C6CF2D813E813227F9
:105CB000232732274C816B818A810E940F0EBBCF34
:105CC0000E942D14B8CF8A81893009F0B4CF8B811E
:105CD000E5E08E9FC00111246FEF70E00BD5862F99
:105CE0000E940A08A8CF8A81893029F08A3009F0F9
:105CF000A2CF1B82A0CF8091C403869586958695FE
:105D0000F3E38F9FC001112486CF84EC93E00E94BF
:105D1000090E91CF80E18A838ECF1A8285E67BCFF0
:105D20008C818D3108F087CF8A809B8098248924CC
:105D30009824A12CB12C8E010F5F1F4F7801E80E23
:105D4000F11CE016F10609F476CF80E025E6821614
:105D50009104A104B10420F4C40185569C4FADD533
:105D6000D80114968C930F5F1F4FBFEF8B1A9B0ABD
:105D7000AB0ABB0AE6CF8091A4029091A502892BC1
:105D800009F459CF8C818D3108F055CF882E912C94
:105D9000A12CB12CCA80DB80DC24CD24DC24E12CB6
:105DA000F12C8E010F5F1F4F412C512C32014814F2
:105DB00059046A047B0408F03ECFE5E6CE16D10410
:105DC000E104F10438F4D80114966C91C6018556AB
:105DD0009C4F8FD5BFEF4B1A5B0A6B0A7B0AEFEF24
:105DE000CE1ADE0AEE0AFE0A0F5F1F4FE0CF0E94B6
:105DF000561621CF83E08FCF8C818D3108F01BCFD9
:105E0000882E912CA12CB12CCA80DB80DC24CD24DF
:105E1000DC24E12CF12C412C512C32018E010B5F42
:105E20001F4F481459046A047B0408F004CF80E033
:105E3000F2E5CF16F2E0DF06E104F10418F4C60142
:105E400089963BD5D8018D938D01BFEF4B1A5B0A24
:105E50006B0A7B0AEFEFCE1ADE0AEE0AFE0AE1CFEA
:105E60002C81022F10E02D3108F0E5CE8A819B8134
:105E70009827892798272C01612C712C8235F2E014
:105E80009F0708F0D8CE822E912CA12CB12C42E590
:105E900052E060E070E0441955096609770942173D
:105EA00051056105710508F4C6CE2091A402309118
:105EB000A502232B09F03EC01C0129E2220E311C51
:105EC00080FBEE24FF24E0F880FF0BC08896F5D419
:105ED0009D8189279827892781159C4711F48FEF89
:105EE0008D83D501C401840D951DA61DB71D80FFAE
:105EF00019C0680141E0C41AD108CE0105968C0D85
:105F00009D1D9CA78BA7C101800F911FD6D4ABA567
:105F1000BCA59C9181159C4721F48FEFEBA5FCA5B6
:105F200080838601FE013196EE0DFF1D2FEFE016F6
:105F3000F10638F08E010F5F1F4FC12CD12C760176
:105F400025C09481858181159C4711F42483258384
:105F500042E0E40EF11C3296EACF82E5481682E078
:105F600058066104710430F4D80114966C91C20192
:105F70008996BFD4BFEFCB1ADB0AEB0AFB0AEFEF1F
:105F80004E1A5E0A6E0A7E0A0F5F1F4FC814D904AC
:105F9000EA04FB0410F34FCE8091A4029091A50275
:105FA000892B09F448CECE0101960E94B00CFFEF78
:105FB00021EE34E0F15020403040E1F700C0000015
:105FC0006CCB88E0E2E1F1E0DE01919601900D9268
:105FD0008A95E1F7FE0132968FE1DF011D928A95E5
:105FE000E9F786E0898388E07F96DE0115960190C7
:105FF0000D928A95E1F71FCE88E4898382E08A8337
:106000001B821C8218CE8B819C81092E000CAA0B4E
:10601000BB0B25E0880F991FAA1FBB1F2A95D1F73C
:10602000AC01BD01405E5F4F6F4F7F4F481759076E
:106030006A077B0708F4FFCD8834E2E09E07A105DC
:10604000B10508F0F8CD4934F2E05F07610571054C
:1060500020F048E452E060E070E0481B590BBC01BE
:106060006F587A4FCE010196FBD3E5CD4AE150E05F
:106070006FEF70E0CE01079609D48091A402898366
:10608000EA821B821C8281E08D831E82D4CD81E056
:1060900090E09093AA028093A90282E390E090930B
:1060A0008D0280938C020E94440A90938B0280930D
:1060B0008A02C1CDE114F104A1F100918E02109188
:1060C0008F02C0909002D0909102A0908A02B0906E
:1060D0008B020E94440A8A199B098536910540F17A
:1060E0000C211D2100FF24C00E94440A90938B02C2
:1060F00080938A0280918C0290918D0201979093F7
:106100008D0280938C02892B61F41092AA02109266
:10611000A90281E090E09093A5028093A402E12C73
:10612000F12C8091A4028983EA8280918C0273CD44
:1061300082E390E090938D0280938C02F2CF1092D4
:10614000A5021092A40277CD40E250E06FEF70E01C
:10615000CE0101969BD36FCDEB81E93008F06BCD7A
:10616000F0E0ED5DFA4C0FC3FE0135968BE1DF01E7
:106170001D928A95E9F788E089838A838B838C83D3
:1061800083E088A358CD8C819AE0F92E8E010F5DB3
:106190001F4FF8012F2D11922A95E9F7B8010E949F
:1061A000C6158983F801DE01129601900D92FA94CA
:1061B000E1F741CD1C818AE0FE013596DE01919622
:1061C00001900D928A95E1F789A19AA10E941F087A
:1061D0009AA389A38BA19CA10E941F089CA38BA3B7
:1061E0008DA19EA10E941F089EA38DA38FA198A59B
:1061F0000E941F0898A78FA38FEF183060F43AE031
:10620000139FB001112465587D4F4AE050E0CE0144
:1062100081968DD380E089830E942C080CCD2C813F
:106220006AE0CE018196DC01E62F1D92EA95E9F73E
:10623000283008F044C0629FB001112465537D4F9F
:106240004AE050E02AD380E089838AE0FE01B196DB
:10625000DE011296CCCE1C818AE0FE013596DE016D
:10626000919601900D928A95E1F789A59AA50E94D1
:106270001F089AA789A78FEF183060F4FAE01F9FD4
:10628000B001112465537D4F4AE050E0CE01819664
:106290004ED380E089830E94C314CDCC2C816AE068
:1062A000CE018196DC01E62F1D92EA95E9F72830B0
:1062B00030F4629FB0011124655E7C4FC1CF8FEF37
:1062C000C3CF1C818AE0FE013596DE0191960190D4
:1062D0000D928A95E1F78BA19CA10E941F089CA3B7
:1062E0008BA38FEF183060F4FAE01F9FB0011124E8
:1062F000655E7C4F4AE050E0CE01819618D380E085
:1063000089830E94071597CC2C8166E0CE01819687
:10631000DC01E62F1D92EA95E9F7283060F4629FD0
:10632000B001112465597C4F46E050E0B6D280E0C0
:10633000898386E08BCF8FEFFBCF1C8186E0FE0147
:106340003596DE01919601900D928A95E1F789A12B
:106350009AA10E941F089AA389A38BA19CA10E94C5
:106360001F089CA38BA38FEF183060F4F6E01F9FEB
:10637000B001112465597C4F46E050E0CE01819672
:10638000D6D280E089830E94861555CC2B3031050A
:1063900008F068CB95CB2B30310508F01DCB4ACBEC
:1063A00080916502811509F4A2C930E139BD42E14D
:1063B00049BD09B400FEFDCF8091D8008F7D809348
:1063C000D8008091E00082608093E0008091E0003E
:1063D00081FDFCCF0E946D0F8AC91F921FB61F92CC
:1063E00011248F939F93AF93BF9380916402811187
:1063F00013C08091EC019091ED01A091EE01B0915C
:10640000EF014196A11DB11D8093EC019093ED0128
:10641000A093EE01B093EF01BF91AF919F918F9147
:106420001F901FBE1F90189578941F921FB61F9241
:1064300011248F939F93AF93BF938091EC01909120
:10644000ED01A091EE01B091EF010196A11DB11DEA
:106450008093EC019093ED01A093EE01B093EF01D6
:10646000BF91AF919F918F911F901FBE1F90189564
:106470001F920F920FB60F9211242F933F934F93B9
:106480005F936F937F938F939F93AF93BF93EF939C
:10649000FF938091E10082FF09C08091E20082FFBA
:1064A00005C08091E1008B7F8093E1008091DA004C
:1064B00080FF24C08091D80080FF20C08091DA0046
:1064C0008E7F8093DA008091D90080FFA9C080E19F
:1064D00089BD82E189BD09B400FEFDCF81E08093D2
:1064E000A6028091DB01811109C00E94910C0E94DB
:1064F000EE0C8091E20084608093E2008091E100E4
:1065000080FF1AC08091E20080FF16C08091E200F7
:106510008E7F8093E2008091E20080618093E200B0
:106520008091D80080628093D80019BC85E0809368
:10653000A60283E080930F018091E10084FF2FC0C9
:106540008091E20084FF2BC080E189BD82E189BD9A
:1065500009B400FEFDCF8091D8008F7D8093D800D4
:106560008091E1008F7E8093E1008091E2008F7E38
:106570008093E2008091E20081608093E20080914C
:10658000DA01811509F452C084E08093A60280915B
:10659000A602843009F052C082E080930F018091FE
:1065A000E10083FF2CC08091E20083FF28C080912E
:1065B000E100877F8093E10082E08093A602109241
:1065C000DA018091E1008E7F8093E1008091E2000A
:1065D0008E7F8093E2008091E20080618093E200F0
:1065E00042E060E080E00E94BE0C8091F000886094
:1065F0008093F00081E080930F0180930E01FF9162
:10660000EF91BF91AF919F918F917F916F915F912A
:106610004F913F912F910F900FBE0F901F901895A3
:1066200019BC1092A6021092DB0168CF8091E300A2
:1066300087FF02C083E0A9CF81E0A7CF81E0ADCF83
:106640001F920F920FB60F921124EF92FF920F93A9
:106650001F932F933F934F935F936F937F938F93EA
:106660009F93AF93BF93CF93EF93FF9309EE10E007
:10667000F8018081C091EC008F70C795CC27C79539
:10668000C82B108280EFE82EF12CF7018081877FE4
:10669000808378940E94AE0FF8011082F701808108
:1066A00088608083CF70F801C083FF91EF91CF9114
:1066B000BF91AF919F918F917F916F915F914F911A
:1066C0003F912F911F910F91FF90EF900F900FBE70
:1066D0000F901F901895DB018F939F9380D0BF91EF
:1066E000AF91A29F800D911DA39F900DB29F900D21
:1066F00011240895AA1BBB1B51E107C0AA1FBB1F91
:10670000A617B70710F0A61BB70B881F991F5A953D
:10671000A9F780959095BC01CD01089597FB072EB0
:1067200016F4009406D077FD08D0E4DF07FC05D00E
:106730003EF4909581959F4F0895709561957F4F98
:106740000895A1E21A2EAA1BBB1BFD010DC0AA1FB2
:10675000BB1FEE1FFF1FA217B307E407F50720F0CA
:10676000A21BB30BE40BF50B661F771F881F991F45
:106770001A9469F760957095809590959B01AC018E
:10678000BD01CF010895EE0FFF1F0590F491E02D9C
:106790000994082E817006940694811D0694811D2B
:1067A0000694811D0694811D0694811D0694801D0A
:1067B00008956927962769277827872778270895D6
:1067C000A29FB001B39FC001A39F700D811D112432
:1067D000911DB29F700D811D1124911D0895F0DF50
:1067E000A59F900DB49F900DA49F800D911D112425
:1067F00008952F923F924F925F926F927F928F9265
:106800009F92AF92BF92CF92DF92EF92FF920F933F
:106810001F93CF93DF93CDB7DEB7CA1BDB0B0FB649
:10682000F894DEBF0FBECDBF09942A883988488806
:106830005F846E847D848C849B84AA84B984C8849C
:10684000DF80EE80FD800C811B81AA81B981CE0F93
:10685000D11D0FB6F894DEBF0FBECDBFED01089578
:10686000FB01DC0102C005900D9241505040D8F769
:106870000895FB01DC0104C08D910190801921F481
:1068800041505040C8F7881B990B0895DC0101C0A6
:106890006D9341505040E0F70895DC01CB01FC01BD
:1068A000F999FECF06C0F2BDE1BDF89A319600B469
:1068B0000D9241505040B8F70895F999FECF92BD1E
:1068C00081BDF89A992780B50895A8E1B0E042E02B
:1068D00050E0E5CFDC01A40FB51F4150504040F01F
:1068E000CB01840F951F2E9105D041505040D8F711
:1068F0000895262FF999FECF92BD81BDF89A019790
:1069000000B4021639F01FBA20BD0FB6F894FA9AF7
:10691000F99A0FBE08950396272FECDFEADF252FA3
:10692000E9DF242FE7CF0196272FE4DFE2CFDC0158
:10693000CB0102C02D9105D041505040D8F70895A9
:10694000262FF999FECF1FBA92BD81BD20BD0FB68B
:10695000F894FA9AF99A0FBE01960895F894FFCF29
:10696000EC0AF10AF30AF80A080B080B080B080BEB
:10697000080B080B080B080BFA0AFE0A010B060BA2
:10698000160B1C0B200B8B10B110B710B110B710E9
:1069900009112A11B71030123D12C31E2B1FCB1E36
:1069A000951E991ECF1E9D1ED31EDF1EA91E241FDD
:1069B000AD1EE31EB11EE71E0C1FB51EEB1E131FFE
:1069C000BB1EF11EF91EA11ED71EA51EDB1EBF1E7B
:1069D000F51E031F1C1F221F8F1EC71E321F611EA4
:1069E000671E531E5B1E6D1E731E791E8F208F2027
:1069F000C620C62077219221EA20EA2097210E2284
:106A00001F221F22E12FFC2F03301B2E1B2E36309E
:106A100047305A309F30A4301B2E1B2E1B2EAC301B
:106A2000092E0D2E3E2E4A2E552E602E632E732ECD
:106A3000852E062ECC2F8A2E8D2E902EBB2EF72E35
:106A4000FA2EFC2E302FB430C330DA300F312B3118
:086A50004E31613184319D31AA
:106A5800410ACD0DE30DE80DED0DC40D0000010058
:106A680001012431A194477F9D0A004422B6840184
:106A78006201AC008A02A302C3029091929395949A
:106A8800969734C63031323337F7F6F5F4F1E20031
:106A9800E900EA00B500B600B700CD008301CC00DC
:106AA8008A0192019401210223022402250226026E
:106AB80027022A02B300B4006F0070009F01CB01C7
:106AC8009F02A002E200E900EA00B500B600B700A4
:106AD800CD008301CC008A01920194012102230296
:106AE80024022502260227022A02B300B4006F00FE
:0A6AF80070009F01CB019F02A00275
:00000001FF
